:100000000C9466000C9487000C9487000C94870075
:100010000C9487000C9487000C9487000C94870044
:100020000C9487000C9487000C9487000C94870034
:100030000C9487000C9487000C9487000C94870024
:100040000C9487000C9487000C9487000C94870014
:100050000C9487000C94ED0C0C9487000C94870092
:100060000C9487000C94AA110C9487000C948700C0
:100070000C9487000C9487000C9487000C948700E4
:100080000C9487000C9487000C9487000C94C30D8B
:100090000C947D190C9487000C9487000C948700B5
:1000A0000C9487000C9487000C9487000C948700B4
:1000B0000C9487000C9487000C9487000C948700A4
:1000C0000C9487000C9487000C94870011241FBEA9
:1000D000CFEFD1E2DEBFCDBF00E00CBF14E0A0E067
:1000E000B2E0E0EFFBE800E00BBF02C007900D922A
:1000F000AE32B107D9F717E0AEE2B4E001C01D920D
:10010000A831B107E1F70E94B9030C94F6450C94AD
:100110000000109234048091340480933304809161
:10012000330480933204809132048093310410921E
:1001300035040895EEE6F0E080818260808383E0FC
:1001400084BD85BD8AEF87BD0895E1E7F0E0808139
:1001500081608083089580917100817008958091FD
:100160008B04982F9295969596959370282F221F21
:100170002227221F9227282F22952F709227282F7F
:100180002695269592279170880F892B80938B0452
:100190000895909381048093800485EB9BE3909372
:1001A00093048093920483E393E190939904809362
:1001B000980485E694ED90938F0480938E040895BF
:1001C0008091800490918104AC01440F452F441F1D
:1001D000550B5195482759276091920470919304CB
:1001E00070938104609380048091980490919904A5
:1001F000909393048093920420918E0430918F0405
:100200003093990420939804C9010024969587950A
:100210000794969587950794982F802D822793278A
:1002200084279527542F44275295550F507E8427B5
:10023000952790938F0480938E04660F771F6F5FCE
:100240007F4F869F9001879F300D969F300D112420
:10025000C9010895FC019081992351F08091C80053
:1002600085FFFCCF9093CE00319690819923B1F712
:1002700008951F93CF93DF93182F492FE0E1F7E202
:10028000C0E0D0E0812F942FBF010E94AD459B01BB
:100290006115710589F5812F942FBF010E94AD452D
:1002A000182F492FCF016AE070E00E94AD45FB0195
:1002B0002196C430D10531F73097A1F18091C80063
:1002C00085FFFCCF812F942FBF010E94AD45605D5B
:1002D0006093CE00CF016AE070E00E94AD459B01C3
:1002E00061157105F9F0812F942FBF010E94AD4572
:1002F000182F492FF901E2CF8091C80085FFFCCF6C
:10030000822F805D8093CE00812F942FBF010E94A9
:10031000AD45182F492FCF016AE070E00E94AD452E
:10032000FB01CACFDF91CF911F910895982F9F7045
:100330009A3040F48091C80085FFFCCF905D909387
:10034000CE0008958091C80085FFFCCF995C909302
:10035000CE000895CF93DF93EC01892F99278295E2
:100360008F700097C1F48D2F9927009789F4CE01E3
:10037000929582958F7089279F708927009711F039
:100380000E9496018C2F0E949601DF91CF910895D3
:100390000E949601ECCF0E949601E5CF982F8091A4
:1003A000C80085FFFCCF9093CE0080E090E00895D8
:1003B0002091C800332727FD30952227330F221FB5
:1003C0003327C90108958091C80087FFFCCF809131
:1003D000CE0090E008959C018FEF8093850493E018
:1003E000283E390768F5809382048093830424367D
:1003F0003105D8F0C90164E670E00E94AD45609314
:100400008204C9016AE070E00E94AD45CB016AE058
:1004100070E00E94AD4580938304C9016AE070E0FA
:100420000E94AD458093840408952A30310548F731
:10043000C9016AE070E00E94AD458093840408958C
:100440001092820410928304109284040895909173
:100450003604936090933604809337040895809116
:1004600036048360809336040895F999FECF92BDD7
:1004700081BDF89A30B5F999FECF019692BD81BD44
:10048000F89A20B5932F80E030E0282B392BC90152
:100490000895F999FECF92BD81BDF89A80B508956F
:1004A000F999FECF92BD81BD60BDF894FA9AF99A90
:1004B00078940895FF920F931F938C01F62E672F67
:1004C0000E945002C80101966F2D0E9450021F9198
:1004D0000F91FF9008958091C90088618093C900B1
:1004E00083E38093CC001092CD008091C80087FDFB
:1004F00032C08091C90080688093C9008091C1009A
:1005000088698093C1008FE18093C4001092C50078
:1005100090EC91B98CE382B987E384B995B99FEFE8
:1005200097B988EF8AB98BE08BB982E08DB99EB913
:1005300010BA91BB13BA94BB8DB581608DBD81E5B6
:100540008CBD08958091CE008AE00E94FB0D8091C1
:10055000C80087FFCECF8091C80087FDF3CF809180
:10056000C80087FFF8CFEECFEF92FF920F931F9353
:10057000CF93DF93EC0181E0CD32D80750F5C8323C
:10058000D105B0F588E290E090937D0480937C04DF
:1005900090938A04809389040E94381924E234EFEE
:1005A00030938D0420938C0482E08093910080919D
:1005B0008C0490918D04909581959F4F90938D041C
:1005C00080938C04DF91CF911F910F91FF90EF905A
:1005D00008958CE291E090937D0480937C04909345
:1005E0008A04809389040E9438192DE830E2D8CF1C
:1005F000D0937D04C0937C04D0938A04C093890473
:10060000CE010E9438199E0140E050E060E070E7A2
:1006100088E399E30E94D445B901CA01969587956C
:10062000779567959695879577956795969587952C
:100630007795679526E030E040E050E00E94D44591
:1006400079018A01C801AA27BB279C01887F892BD1
:1006500009F45FC0C901807F892B99F0C901807EB0
:10066000892BF1F0C901807C892B49F1C901807087
:10067000892BA1F120703C7F232BE1F11092910096
:1006800096CFF4E016950795F794E794FA95D1F78D
:10069000F0928D04E0928C0486E08093910087CFE5
:1006A000E5E016950795F794E794EA95D1F7F0926F
:1006B0008D04E0928C0487E08093910078CF76E0FF
:1006C00016950795F794E7947A95D1F7F0928D04F3
:1006D000E0928C0483E08093910069CFBB27A12F27
:1006E000902F8F2D90938D0480938C0484E08093C1
:1006F00091005DCF5AE016950795F794E7945A95C7
:10070000D1F7F0928D04E0928C0485E08093910003
:100710004ECFA3E016950795F794E794AA95D1F7E5
:1007200097013ECF85E090E00E9435020E94B4021E
:1007300080918C0490918D0490937F0480937E042B
:1007400010922F04E1E7F0E0808181608083809146
:100750007C0490917D04909391048093900408957B
:1007600085E20E945E15E1E7F0E080818E7F808364
:100770000895AF92BF92CF92DF92EF92FF920F93C4
:100780001F93DF93CF93CDB7DEB760970FB6F89482
:10079000DEBF0FBECDBF0E946B020E94920380910C
:1007A0006E00826080936E0083E084BD85BD8AEF19
:1007B00087BD8BE696E09093AE068093AD06F999DF
:1007C000FECF82E090E092BD81BDF89A80B5982F6F
:1007D000937090932E048295817080936A04F999A6
:1007E000FECF87E090E092BD81BDF89A80B5882366
:1007F00011F0813208F080E180930002F999FECF78
:1008000083E090E092BD81BDF89A80B58F708093AF
:10081000AD04F999FECF84E090E092BD81BDF89AD5
:1008200080B58F7080939A0488E090E00E94350232
:1008300080938B0420917C0430917D04280F391F14
:10084000309381042093800485EB9BE39093930481
:100850008093920483E393E19093990480939804A6
:1008600085E694ED90938F0480938E040E94E000BF
:100870000E94E0000E94E000BC0188E090E00E943D
:100880005A02F999FECF8AE090E092BD81BDF89AB4
:1008900090B5892F8F708093940480919404833055
:1008A00010F01092940492959F709F5F909397041C
:1008B00080919704823008F4E2C00E94BC2C7894A6
:1008C00000E010E01DC08091DA040E94F8150E943B
:1008D0002A17C801849668E270E00E94C1450E9410
:1008E000C0180E945E1580E10E94FB0DC801877050
:1008F0009070892B69F00F5F1F4F0C32110579F052
:10090000083208F7802F0E94C0180E942615DBCFFE
:100910000E9479140F5F1F4F0C32110589F70E9456
:10092000D5150E942A170E94791480E00E94B41203
:10093000882331F083E00E94B412882309F0EBC0D1
:1009400083E00E94B412882309F09DC08091DA04EC
:100950008093C40610920507109298051092210604
:1009600081E080932706109228068091C40660914A
:10097000050740912106209127060BE616E00E940C
:10098000C22B60912106C8010E94F3280E947E2894
:100990000E9479148091360483608093360410920B
:1009A00037048091D504873009F466C0883030F56B
:1009B000823009F449C08330A8F5882309F44AC07D
:1009C000813009F444C00E9479140E947E28882353
:1009D000F9F68091D5048630B1F781E00E94E012EB
:1009E000882389F380E00E94B412882361F30E9477
:1009F000D5150E942A17E0E0F0EF19948C30C9F168
:100A00008D3038F4883061F18B30E9F60E940B228A
:100A1000BFCF8E3011F18E30A0F08F30A1F60E9442
:100A2000D22CB6CF843051F0843028F0853059F67E
:100A30000E94D531ADCF0E949C24AACF0E94B11C48
:100A4000A7CF0E946A44A4CF0E94EA3BA1CF0E9494
:100A5000053E9ECF0E9443119BCF0E94131998CF51
:100A60000E94D5150E9479140E947E288823D1F314
:100A70008FCF0E94C10F8CCF0E94532689CF82E076
:100A8000809397041ACF8CE00E94B412882309F453
:100A90005DCF7E010894E11CF11CBB2491E1C92EBD
:100AA000D12CCC0EDD1E8FE0A82E87010E94E00025
:100AB000F801908381830E5F1F4F0C151D05B1F760
:100AC000F70104C031960E171F0791F02081822F85
:100AD00090E08F7090700D9724F0822F8F7080833C
:100AE000282F2D3079F78E2F8E198F3009F072C094
:100AF00080E060E04B2D21E087010E94372C85E5E6
:100B00000E94DF180E942A17B394F0E8BF1669F616
:100B10000E94D5151BCF10922E0410926A0460918A
:100B20006A0470E06170707062957295707F7627CC
:100B3000607F762782E090E00E9450020E94BC2CE9
:100B40001092AD0410929A0483E090E060E00E945D
:100B5000500284E090E060919A040E94500288E77D
:100B600090E090937D0480937C0485E090E068E7BA
:100B700070E00E945A0280E18093000260910002BE
:100B800087E090E00E9450021092940488E08093E5
:100B90009704809197046091940490E00197829566
:100BA0009295907F9827807F9827682B8AE090E025
:100BB0000E94500210E082E20E94921583E20E949D
:100BC00092150E942A1782E30E94FB0D1F5F1832C4
:100BD00091F79ECFA08276CFCF92DF92EF92FF92D5
:100BE0000F931F93CF93DF93F89480912E0481305D
:100BF00009F4C6C280917304813009F4F2C1809176
:100C00003104863060F010923104809132048F5F9D
:100C100080933204809133048F5F809333048091FA
:100C20003304882341F08091330490E08370907006
:100C3000892B09F4BFC180913404883038F01092B8
:100C4000340480912E04882309F493C180913304E5
:100C50008F70809333049091320480910002981732
:100C6000C0F010923204809135048F5F8093350478
:100C70009091350480919704981708F077C180917E
:100C8000360482608093360480913A0481608093B8
:100C90003A0480911207882329F480913204882332
:100CA00009F45AC180913204882329F48091730495
:100CB000823009F442C28091D5048C3009F480C19D
:100CC00080912E04882301F5909143048091E903DB
:100CD000981710F0109243048091430480FF40C2A3
:100CE0005C988091430480FF0FC0809143048F5F24
:100CF000809343047894DF91CF911F910F91FF90DF
:100D0000EF90DF90CF900895809174042091E903D3
:100D10004091E90390E030E0240F311D82179307E2
:100D200014F010927404809174046091E903669544
:100D30000E94A145992309F48AC0DD248091D5043D
:100D4000873009F490C0883008F068C1813008F01D
:100D50000CC280917304823009F438C2809112076A
:100D6000882321F082E0D81609F43BC28091120753
:100D7000882309F401C2809160048F70809360041D
:100D80008091330490E08370907002970CF4B4C1AA
:100D900085E20E945E158091600490E083709070FF
:100DA00002970CF4A6C18FEF8093580480916904D8
:100DB000882309F06EC180917204882329F0809104
:100DC0003704882309F09CC180913804882309F0F6
:100DD0004EC10E942A17DD2031F080912F048F5FD1
:100DE000817080932F042091890430918A0480912E
:100DF0007C0490917D042817390719F0C9010E94DD
:100E0000B402809174048F5F80937404809106070C
:100E10008F5F80930607809131048F5F8093310448
:100E2000809143048F5F8093430420910607809153
:100E3000E90330E0869586954CE0849FC00111243B
:100E40002817390714F010920607789454CF809130
:100E50002F04882309F46EC1DD24D3948091D50436
:100E6000873009F070CF81E0D81609F49CC2E2E027
:100E7000DE1609F06ECF809160048F5F809360046E
:100E800080911207882309F461C080919905882315
:100E900009F51092060780919D05882349F48091F9
:100EA0000807882329F080916904882309F044C544
:100EB0008091210660916906680F8091AD0690913E
:100EC000AE060E94F3281092600480916404882387
:100ED00009F47FC480919905E091AD06F091AE06CA
:100EE000E80FF11D808180937B04809188048093BA
:100EF000860480917B0480748093880480916904C7
:100F0000882309F0E4C380917B048F708F3009F44B
:100F100054C480917B048F708F3071F080917B047A
:100F20000E9417299091B3066091860440917B043A
:100F30004078890F0E94921C8091D504833009F477
:100F4000F3C38091D504873009F4D0C3809136046F
:100F5000816080933604FDCE80917304823009F065
:100F6000A1CE109273040E94EA2F9CCE10923504F9
:100F700086CE20917C0430917D04809190049091E4
:100F800091042817390709F461CE8091120788234C
:100F900009F05CCE85E20E94261560917C04709178
:100FA0007D04709391046093900485E090E00E942A
:100FB0005A024CCE809134048F5F809334043BCE30
:100FC00080913A0480FF0AC080911207882309F0BB
:100FD00090C180913F04882309F0ECC210923A043A
:100FE0006FCE80911207882309F0B5C00E94EA2FC6
:100FF00080912E04882309F0B0C0109234048091AF
:1010000034048093330480913304809332048091BC
:10101000320480933104109235049FC08B3009F460
:1010200022CF8C3008F0E1C0883009F092CEF1E098
:10103000DF1609F41AC382E0D81609F08ACE80912F
:101040007A04809330048091790480937A040E941A
:10105000AF008093790480917A048F7360E040E060
:101060000E94921C80917A040E94BA0E72CE0E9455
:10107000D1188091330480FDACCEE0913304E69525
:10108000F0E0E370F070EE57FB4F80810E94C618CD
:10109000A0CE8CE20E941729982F809160048111C4
:1010A000945F80910607882341F480916A04882325
:1010B00009F4D5C283E20E9426158091060782308A
:1010C00009F079CE80916A04882379F480916704CD
:1010D000823008F4E7C2809125060E9417294091CA
:1010E0002506407860E00E94921C83E20E945E1513
:1010F00062CE109258045ACE85E20E9426154BCE3D
:1011000080919404813009F43EC180919404882335
:1011100009F05ACE8091360480FF56CE8091360475
:101120008E7F809336040E94EA15809199050E9473
:10113000F8154ACEB2E0DB2E01CE8091D504853081
:1011400009F4B9CD1092740410922F0410929905ED
:1011500010927304B0CD0E94BE2F109273044FCD35
:101160005C9A88EF0E94210FBCCD843008F47BCEBE
:10117000853009F0EECD77CE81E20E945E15FBCD81
:101180000E9445128823A9F080917204882309F0F7
:1011900076C2109234048091340480933304809199
:1011A000330480933204809132048093310410928E
:1011B00035040E945712882309F41CCD80917204D3
:1011C000882309F417CD0E94BE2F14CD81E20E941E
:1011D0005E158091310463E00E94A145992309F0D6
:1011E000CACD81E20E942615C6CD8C3021F08D300B
:1011F00009F0AFCD38CE0E94EA1580913A0480FD07
:10120000D5C180913F04882309F0CAC1E1E0DE1610
:1012100009F459C1F2E0DF1609F09BCD809160041A
:101220008F5F8093600480911207882309F491CD29
:10123000E0916906F0E0E155F94F808184FD3DC2FF
:1012400086E08093E90380919905E091AD06F091E5
:10125000AE06E80FF11D808180937B0480918804A5
:101260008093860480917B048074809388048091AD
:101270007B048F708F3009F422C280917B048F70C1
:101280008F3071F080917B040E9417299091B306F2
:101290006091860440917B044078890F0E94921CE3
:1012A00080913904982F92959F709093C406982F3F
:1012B0009770909321068695869586958170809388
:1012C000050780910507882309F0F0C188E00E9496
:1012D000261581E00E945E150E94D316809121069A
:1012E0008F5F0E947316809112078170809312079E
:1012F00030CD80911207823008F470CE80913F0487
:10130000882329F480918505882309F467CE80918C
:10131000400480933904909169069F5F9093690619
:10132000909169069170909369066091690670E0EA
:1013300062957295707F7627607F76276559794F21
:101340007093AE066093AD0690916906C92FD0E008
:101350000E94652BC155D94F8883E0916906F0E062
:10136000E155F94F80818F708F5F8093EB03E0919F
:101370006906F0E0E155F94F808184FD7EC186E089
:101380008093E9032BCE8091360481FFBECE8091FD
:1013900036048D7F809336040E94EA1580913504CF
:1013A0000E94F815B2CE80919D058F5F80939D05B8
:1013B00080911207882309F4CCCC809199058F5F26
:1013C00080939905909199058091EB03981710F0FF
:1013D0001092990580919905882309F06EC080913B
:1013E000D504833009F420C110E08091D504873002
:1013F00009F4A7C181E00E94C228809169068F5F2D
:1014000080936906C09069069091690680912706CD
:10141000981708F443C080916404882319F481E08C
:10142000809371048091D504813009F4E5C18091E5
:10143000D504823009F4DCC182E00E94C2281092F7
:101440009D0580916904882369F0809167048093E9
:10145000080780910807882329F01092670481E02B
:1014600080939705109269068091D504833009F422
:1014700000C28091D504873009F4D5C18091280637
:10148000882309F0BCC190910507809198059817B1
:1014900029F080916404823008F482C28091690648
:1014A00090E082959295907F9827807F9827855924
:1014B000994F9093AE068093AD068091690488237E
:1014C00009F047CC57C080911207882309F441CC1A
:1014D000809199058F5F8093990580913F048823BF
:1014E00009F4D0C090914004809139048917D1F15A
:1014F000F0906906F394FE220F2D10E0E801C295EA
:10150000D295D07FDC27C07FDC27C559D94F809189
:101510004004BE010E94652B0155194FF8018083DC
:10152000E0916906F0E0E155F94F2081F8018081F2
:1015300090E030E08227932784FD14C0809140041E
:1015400080933904F0926906E0916906F0E0E15574
:10155000F94F80818F708F5F8093EB03D093AE063D
:10156000C093AD06809199056091EB030E94A1455F
:101570009093990580919905E091AD06F091AE06A2
:10158000E80FF11D808180937B0480917B048F7034
:101590008F3009F47FC0809188040E94A91CD9CBA8
:1015A00080913F0481500E94F81530CE8FE00E9458
:1015B000F81527CE80914004809339040E94EA2FC9
:1015C00080912E04882381F4109234048091340495
:1015D00080933304809133048093320480913204E9
:1015E0008093310410923504809169068F5F809357
:1015F0006906809169068170809369066091690629
:1016000070E062957295707F7627607F76276559C6
:10161000794F7093AE066093AD0680916906C82F2E
:10162000D0E08091390494CE80918105909182051B
:1016300001969093820580938105209181053091D8
:10164000820580918C0590918D052817390708F443
:10165000CBCE109282051092810511E0C6CE892F63
:1016600060E040E00E94921C25CD80E00E94A91C11
:1016700080917A040E94F90E6CCB88E081CE0E94A2
:10168000EA2F87CD80918505882309F06BCF0E94D2
:10169000BE2F68CF80918804882309F096C01092ED
:1016A000880479CF80E00E94A91C1FCD88E00E94A9
:1016B0005E1581E00E9426150FCE88E0C2CD809194
:1016C0007B048F7080937B0410928804D6CD809128
:1016D00021066091270640919A05209128060091E5
:1016E0009E05E09098050E94191826CC8091380438
:1016F000813009F419C18091810590918205E091B2
:101700009205F0E0EE0FFF1FEF5FFD4F60817181EA
:1017100082959295907F9827807F98270E94AD456B
:10172000862F0E94031612CC80913804813009F074
:1017300008CC809181059091820501960E94EB0171
:1017400000CC80915F04813009F054CE6091050790
:1017500080912106409169062091B306480F89E8DF
:1017600095E00E940F1E8091920560918105709115
:101770008205409189050E94751E80918105909196
:10178000820501969093820580938105E0919205F0
:101790002091810530918205F0E0EE0FFF1FEF5F91
:1017A000FD4F808191812817390708F423CE1092CC
:1017B0005F0483E20E945E151DCE80917B048F70D2
:1017C00080937B0410928804A4CB81E00E94A91C22
:1017D00066CF809121066091270640919A0520915D
:1017E000280600919E05E09098050E94191872CB7A
:1017F00081E08093710420CE8093710418CE0E9402
:10180000AF2880916404823008F048CE8091C406ED
:101810006091050740912106209127060BE616E00E
:101820000E94C22B3BCE80915F04813009F026CE0E
:1018300080918505882309F0B8C0809186058823AA
:1018400009F41CCE10928605809192056091810565
:10185000709182056C190E943C1E809192050E9435
:10186000CF1E909394058093930580E00E945E15AF
:1018700005CE80918505882309F079C08091860581
:10188000882309F44EC01092820510928105809140
:10189000D00480939205809192050E94D81E909367
:1018A0008D0580938C05809192050E94CF1E9093A8
:1018B0009405809393052091930530919405809130
:1018C0008C0590918D052817390720F0109294050A
:1018D0001092930580918605882309F053C080916A
:1018E000920560918105709182050E94291F809365
:1018F0008905809192056091890540EE55E028E9BF
:1019000035E00AE915E0ECEAEE2EE6E0FE2E0E9454
:10191000EF1D81E0809328068091AC068093B3068A
:10192000A8CD1123B9F2AFCF8091810590918205A6
:1019300001960E94EB01DFCE81E00E94A91C80E0AD
:101940000E94A91C609127068BE696E045EC56E0C4
:101950002FE935E00E94222A109269048AE00E9451
:1019600033291092880482E00E94FB0DA1CA1092D4
:101970008505109282051092810583E20E945E1512
:1019800011E07CCF1092860580919305909194058B
:10199000909382058093810580E00E945E159FCF21
:1019A000809198058093050731CF10925F041092C3
:1019B00085058091920560918105709182050E9454
:1019C0004C1E809192050E94D81E90938D058093A5
:1019D0008C0583E20E945E1530CF1F920F920FB6E6
:1019E0000F920BB60F9211241F932F933F934F9397
:1019F0005F936F937F938F939F93AF93BF93EF9377
:101A0000FF9320B1227090B1809196042817F1F0D5
:101A1000892F8170222309F47AC0882309F47AC0BF
:101A20008091890490918A04019790938A0480930D
:101A3000890431E08D32930708F47AC08CE291E09A
:101A400090938A04809389042093960480914C0497
:101A50008F3F29F080914C048F5F80934C048091DC
:101A60004D048F3F29F080914D048F5F80934D048A
:101A700080917704909178048F5F9F4F49F0809117
:101A8000770490917804019690937804809377047A
:101A900080915B0490915C048F5F9F4F49F080912F
:101AA0005B0490915C04019690935C0480935B04CA
:101AB00010912E04113009F445C080914604909194
:101AC0004704892B81F08091460490914704019747
:101AD0009093470480934604809146049091470474
:101AE000892B09F45C98FF91EF91BF91AF919F9181
:101AF0008F917F916F915F914F913F912F911F91A6
:101B00000F900BBE0F900FBE0F901F90189588235B
:101B100009F486CF8091890490918A04019690936C
:101B20008A048093890431E08D32930708F086CFD0
:101B3000889708F089CF88E290E090938A04809398
:101B4000890482CF99B19295917080914A0488233B
:101B500019F090934A04C7CF9923D9F38091440494
:101B6000909145040196909345048093440410920B
:101B70004504109244040E94EC0588EF0E94210F56
:101B800010934A04B0CF1F920F920FB60F920BB66C
:101B90000F9211242F933F934F935F936F937F93F3
:101BA0008F939F93AF93BF93EF93FF9380917E04A6
:101BB00090917F04909395008093940080918C0481
:101BC00090918D0490937F0480937E040E94EC0595
:101BD000FF91EF91BF91AF919F918F917F916F9105
:101BE0005F914F913F912F910F900BBE0F900FBEC1
:101BF0000F901F90189520EA3FE0E22FF32F3197C6
:101C0000F1F78A95D1F70895882309F41EC09AEF59
:101C100020EA3FE0E22FF32F3197F1F79A95D1F7C1
:101C2000E22FF32F3197F1F79A95D1F7E22FF32FA7
:101C30003197F1F79A95D1F7E22FF32F3197F1F71A
:101C40009A95D1F7815009F0E5CF08951092A30439
:101C50001092AC0408951F93CF93DF93EC01142FDF
:101C60006F777885772309F44CC0462F50E0888140
:101C700090E08F7790704817590779F121E030E0B4
:101C80000DC0D901FE01E20FF31F808190E08F7734
:101C900090702F5F3F4F8417950709F1271788F33E
:101CA000272F2F5F293030F128E0922F822F91507B
:101CB000FE01E80FF11DDE01A90FB11D8C9180839B
:101CC000892F9923A1F71536C0F480E0862B8883ED
:101CD0002887DF91CF911F910895A0E0B0E01536DD
:101CE00070F480E0AC0FBD1F862B8C93DF91CF91F9
:101CF0001F9108952223C9F6E6CF80E8E7CF80E858
:101D0000F1CF91E081E021E0D2CFCF93DF93EC01DE
:101D100038853323B9F06F7770E0888190E08F7752
:101D200090706817790789F0FE0120E008C0818172
:101D300090E08F77907031966817790739F02F5FB0
:101D40002317A8F3DF91CF91089520E0323068F097
:101D5000922F9F5FFE01E20FF11DDE01A90FB11D61
:101D60008C918083292F9317A0F331503887DF910E
:101D7000CF910895282F90919A048091C00085FFFB
:101D8000FCCF90699093C600822F90E08F73907083
:101D9000892BB1F48091C00085FFFCCF1092C60062
:101DA000822F829586958695837080FD19C09091CB
:101DB00023028091C00085FFFCCF9093C600089558
:101DC0008091C00085FFFCCF822F8F73875E809348
:101DD000C600822F829586958695837080FFE7CF17
:101DE000909121028091C00085FFFCCF9093C600A6
:101DF0000895282F90919A048091C00085FFFCCF10
:101E000090689093C600822F90E08F739070892B1A
:101E100039F48091C00085FFFCCF1092C60008C045
:101E20008091C00085FFFCCF2F73275E2093C600F2
:101E3000909122028091C00085FFFCCF9093C60054
:101E40000895982F8091C00085FFFCCF9093C60025
:101E500080E090E00895909141048091420420E058
:101E600030E0981711F021E030E0C9010895909119
:101E70004104809142049817D1F3F8949091410461
:101E8000E92FF0E0E255FB4F80819F5F9093410482
:101E9000909141049F7190934104789490E008954B
:101EA0009091410480914204981729F00E94370FC5
:101EB000482F87FD03C040E0842F0895582F529586
:101EC0005F705F30C9F3282F30E02F703070809141
:101ED000AD0490E02817390771F750933C04ECCF1C
:101EE00090919A048091C00085FFFCCF906B9093F5
:101EF000C6008091C00085FFFCCF8BE78093C600B1
:101F00008091C00085FFFCCF1092C600089580919B
:101F10002E04823049F08091C00085FFFCCF8CEF09
:101F20008093C6000E94700F089590913004891329
:101F3000089580E00E94A91C8FEF809330040895DB
:101F40001F93182F962F6623B9F060E0809130041C
:101F50008F3F09F061E0953648F4812F895140E0C8
:101F60000E94921C109330041F910895812F895173
:101F700041E00E94921CF6CF60E00E94950F1F91F5
:101F80000895FF920F931F93809185058170809330
:101F9000850580918505809372040E94D5158091F6
:101FA0008505882309F02EC10E942A178BE090E056
:101FB0000E944902809324028CE090E00E94490232
:101FC00080932502FF2410E00E9479140E947E284D
:101FD000882309F048C090914104809142049817E9
:101FE00069F00E94370F682F87FD6BC080913C0419
:101FF000883009F4ACC0893009F477C0112371F43A
:102000002091A304222349F48091AC04882329F46D
:1020100080911207882309F4E0C010E087E10E9454
:102020000913882389F2809185058F5F8093850548
:1020300080918505817080938505809185058093C9
:10204000720480E00E945E1580918505882309F462
:10205000BBCF80E00E9426150E9479140E947E2842
:10206000882309F4B8CF0E94700F81E0809327067F
:102070008091050780939805109228068091C406E8
:102080006091050740912106209127060BE616E096
:102090000E94C22B60912106C8010E94F328FF20F4
:1020A00061F08BE090E0609124020E9450028CE08D
:1020B00090E0609125020E9450021F910F91FF90C5
:1020C0000895482F42954F704F3009F498C0282F3B
:1020D00030E02F7030708091AD0490E02817390700
:1020E00009F48DC010923C046FCF67FDBAC0062F73
:1020F0000E94370F482F112309F090CF50912402EE
:10210000051748F0852F90E00F96202F30E08217BA
:1021100093070CF082C050912502051708F470CF88
:10212000852F90E00C96202F30E0821793070CF457
:1021300067CF051B84EA94E0602F0E942B0E8091EC
:10214000A4048F778093B3062091A3045BCF67FD2F
:1021500084C0062F0E94370F112371F5409124028D
:10216000041748F0842F90E00F96202F30E082175C
:1021700093070CF06BC040912502041708F440CF80
:10218000842F90E00C96202F30E0821793070CF4F8
:1021900037CF041B84EA94E0602F0E94850E809163
:1021A000AC04882309F42CCF8091A4048F7780930A
:1021B000B3062091A30426CF113009F456C089E15B
:1021C0000E945E150093250280918505809372041C
:1021D0002091A304FF24F39415CF84E00E940913F7
:1021E0008823A1F485E00E940913882309F415CF00
:1021F0001092720489E10E94261512E00FCF4093DD
:102200003C04F4CE80E00E942615CECE10927204DB
:1022100080E20E94261511E001CF051B8BE994E0B6
:10222000602F0E942B0E2091A30420933F048091E5
:102230009B048F77809340048091DA04909140044E
:102240008295807F890F80934004DCCE041B8BE94C
:1022500094E0602F0E94850EE6CF0E94370F082F72
:1022600079CF0E94370F082F43CF80E20E945E157E
:102270000093240280918505809372042091A30429
:10228000FF24F394BFCE1F930E94EA158091AD0402
:102290000E94F8150E94791484E60E94FB0D0E94AA
:1022A000791484E60E94FB0D0E9479148FEF8093CD
:1022B00030040E9479140E947E28882301F59091B1
:1022C0004104809142049817A1F30E94370F482FD0
:1022D00087FD19C080913C04883039F1893049F775
:1022E00047FD30C0142F0E94370F682F812F0E94A6
:1022F000A00F0E9479140E947E28882301F30E9477
:10230000700F1F910895582F52955F705F30B9F08C
:10231000282F30E02F7030708091AD0490E02817A6
:10232000390769F010923C04C4CF47FD0FC0142F49
:102330000E94370F682F812F0E94950FBACF5093BC
:102340003C04C8CF0E94370F182FCDCF0E94370F03
:10235000182FEECF1F920F920FB60F920BB60F925F
:1023600011242F933F934F935F936F937F938F939A
:102370009F93AF93BF93EF93FF939091C6009A3FC3
:1023800009F442C09C3FA9F1983F09F44AC08091EA
:102390004204E82FF0E0E255FB4F90838F5F80937B
:1023A0004204809142048F718093420490914204D0
:1023B00080914104981751F4809141048F5F80937C
:1023C0004104809141048F7180934104FF91EF910A
:1023D000BF91AF919F918F917F916F915F914F913D
:1023E0003F912F910F900BBE0F900FBE0F901F903B
:1023F000189580917204882349F380912E048230CD
:1024000029F70E94BE2FE2CF80912E048230F1F690
:1024100080917204882311F00E94EA2F0E948900A3
:10242000D5CF809177049091780490932D04809378
:102430002C04109278041092770480912E0482303C
:1024400029F680913D0490913E04019690933E04BC
:1024500080933D045C9A8091C00085FFFCCF88EF9B
:102460008093C6000E94EC0580912C0490912D046D
:102470009695879580934604A9CF5F9A0895809199
:102480002E04813009F05F98089599B1991F99271A
:10249000991F80914804882311F4992321F4909383
:1024A000480480E008959093480481E0089599B12C
:1024B000991F9927991F80914904882311F0992326
:1024C00021F09093490480E008951092490481E03E
:1024D00008958AB1806F8AB98BB18F708BB90895D6
:1024E0008AB18F708AB98BB18F708BB90895AC01A6
:1024F000F89428980000000000000000289A20E0CE
:1025000030E01EBC0DB407FEFDCF8EB5FA01E20F20
:10251000F31F80832F5F3F4F2330310591F778946D
:10252000089516980895169A089520B1269526952F
:102530002F70822F90E02695322F36953695227097
:10254000322B880F991F282F2470322B880F991F48
:10255000880F991F8870382B8FE0831B089580B1F6
:10256000869586958F700895282F883188F4E82FF6
:10257000E695E695E695F0E0E552FB4F808190E028
:10258000277002C0959587952A95E2F78170089586
:1025900080E00895282F883188F4E82FE695E695A5
:1025A000E695F0E0EE52FB4F808190E0277002C08C
:1025B000959587952A95E2F78170089580E00895B2
:1025C000282F883188F4E82FE695E695E695F0E027
:1025D000EA52FB4F808190E0277002C09595879565
:1025E0002A95E2F78170089580E008958091DB04D8
:1025F000882321F48091DC04882319F090E0892F4E
:10260000089590E08091DD048823C9F791E0892F37
:102610000895282F8831A0F4482F46954695469571
:10262000277081E090E0382F01C0330F2A95EAF738
:10263000A42FB0E0FD01EE52FB4F8081832319F4FB
:1026400020E0822F0895232F30E020953095A55269
:10265000BB4F8C9190E028233923232B89F7342F0B
:102660003F5F832F63E00E94A145E92FF0E0E55230
:10267000FB4F8081882321F720E0832F8F5F0E940A
:10268000A145E92FF0E0E552FB4F80818823C9F690
:1026900021E0D7CF1F93CF93DF93C8E3D2E010E0C0
:1026A00088810E94B412882329F41F5F21961D306F
:1026B000B9F71FEF812FDF91CF911F9108951F93DD
:1026C000CF93DF93C8E3D2E010E088810E94CA1262
:1026D000882349F41F5F21961D30B9F780E0DF9110
:1026E000CF911F910895812F8F5FDF91CF911F911F
:1026F00008951F93CF93DF93C8E3D2E010E0888161
:102700000E94E012882349F41F5F21961D30B9F71B
:1027100080E0DF91CF911F910895812F8F5FDF912E
:10272000CF911F9108951F93CF93DF93C0E3D2E021
:1027300010E088810E94B412882349F41F5F21961B
:102740001830B9F780E0DF91CF911F910895812F64
:102750008F5FDF91CF911F9108951F93CF93DF93E8
:10276000C0E3D2E010E088810E94CA12882349F4B5
:102770001F5F21961830B9F780E0DF91CF911F914C
:102780000895812F8F5FDF91CF911F9108951F933F
:10279000CF93DF93C0E3D2E010E088810E94E01283
:1027A000882349F41F5F21961830B9F780E0DF9144
:1027B000CF911F910895812F8F5FDF91CF911F914E
:1027C0000895CF93DF93C0E3D2E088810E94B412D2
:1027D000882349F4219682E0C833D807B1F780E016
:1027E000DF91CF91089581E0DF91CF910895FF921D
:1027F0000F931F93CF93DF93C0E3D2E0FF2400E059
:1028000006C00F5F219682E0C833D80789F018818F
:10281000812F0E94B4128823A1F7812F0E94E01219
:10282000882381F3F394219682E0C833D80779F79F
:1028300081E0F81639F080E0DF91CF911F910F9180
:10284000FF90089580E00730B9F781E0F5CF1F933E
:10285000CF93DF93C6E2D2E010E088810E94CA12D3
:10286000882349F41F5F21961A30B9F780E0DF9181
:10287000CF911F910895812F8F5FDF91CF911F918D
:10288000089580914B0410924B04089580E00895C0
:10289000382F883100F5282F277081E090E0982F9D
:1028A00001C0990F2A95EAF7832F8695869586951C
:1028B000A82FB0E0FD01EE52FB4F8081892369F41F
:1028C000FD01EA52FB4F8081892371F4A552BB4F71
:1028D0008C91982339F480E00895832F0E94F91792
:1028E00082E0089583E00895832F0E94011881E01B
:1028F0000895EF92FF920F931F93DF93CF9300D031
:1029000000D0CDB7DEB71092D2041092D604109248
:10291000D3041092D7041092D4041092D80480915A
:102920004C048A3068F426960FB6F894DEBF0FBECA
:10293000CDBFCF91DF911F910F91FF90EF90089540
:1029400010924C0416987E010894E11CF11CC701FA
:102950000E9477128091DB048C838091DC048D834C
:102960008091DD048E8360E070E001E010E0E62FEE
:10297000E695E695E695F0E0CB01877090709801BA
:1029800002C0220F331F8A95E2F7C901AF014552F9
:102990005B4FD701AE0FBF1F3C91E252FB4F20812E
:1029A000232B28238095FA0130818323282B208331
:1029B0006F5F7F4F68317105D1F60E949512982F95
:1029C00096959093DA048093D004169A40E050E0F4
:1029D000BE016C5F7F4FDA01A252BB4FF701E40FDB
:1029E000F51F80818C93FB01E40FF51F2081FA0114
:1029F000E552FB4F9081FA01EE52FB4F822F8095FA
:102A000089238083FA01EA52FB4F909592239083A9
:102A10004F5F5F4F43305105F1F690B19695969513
:102A20009F708091CE04891721F010924D049093ED
:102A3000CE0480914D048F3630F09093CF04809176
:102A4000CF048093CE040E942A176DCF282F88329E
:102A5000C0F4E82FE695E695E695F0E0277081E072
:102A600090E001C0880F2A95EAF7DF01A25BBB4F17
:102A70002C91282B2C93ED5AFB4F8095208182239B
:102A800080830895282F8832C0F4E82FE695E695D4
:102A9000E695F0E0277081E090E001C0880F2A956C
:102AA000EAF7DF01AD5ABB4F2C91282B2C93E25B48
:102AB000FB4F80952081822380830895282F8832C0
:102AC000C8F4E82FE695E695E695F0E0277081E0FA
:102AD00090E002C0880F991F2A95E2F78095DF01E8
:102AE000A25BBB4F2C9128232C93ED5AFB4F2081E6
:102AF000822380830895282F883298F4E82FE69562
:102B0000E695E695F0E0ED5AFB4F277081E090E006
:102B100002C0880F991F2A95E2F7809520818223B1
:102B200080830895282F883290F4E82FE695E69563
:102B3000E695F0E0E25BFB4F277081E090E002C099
:102B4000880F991F2A95E2F720812827208308956E
:102B5000E82F883298F4282F277081E090E002C097
:102B6000880F991F2A95E2F7E695E695E695F0E03D
:102B7000ED5AFB4F20812823822F089520E0822FD9
:102B80000895982F969596959695EEE4F4E0E90FC2
:102B9000F11D208130E0877002C0359527958A9518
:102BA000E2F721703070C90108951092520410921A
:102BB00051041092500410924F0410924E0410923F
:102BC0005704109256041092550410925404109217
:102BD00053040895CF93DF93C4EAD2E089910E9411
:102BE0005E1582E0C43BD807C9F7DF91CF91089505
:102BF000803108F00895E82FF0E0EC55FD4F80811A
:102C00000E94261508950F931F93CF93DF93082FEB
:102C1000C4EAD2E010E007C088810E9426151F5F39
:102C20002196103149F01017B8F388810E945E1583
:102C30001F5F21961031B9F7DF91CF911F910F914E
:102C40000895803108F00895E82FF0E0EC55FD4F2D
:102C500080810E9442150895803110F080E008952F
:102C6000E82FF0E0EC55FD4F80810E94C1150895DA
:102C7000803110F080E00895E82FF0E0EC55FD4F32
:102C800080810E94A8150895883108F00895E82FE2
:102C9000F0E0E158FD4F80810E94261508958831AB
:102CA00008F00895E82FF0E0E158FD4F80810E9480
:102CB00042150895883108F00895E82FF0E0E158B2
:102CC000FD4F80810E945E150895CF93DF93CFE77B
:102CD000D2E089910E945E1582E0C739D807C9F712
:102CE000DF91CF910895E82F8150883008F0089542
:102CF000F0E0EA58FD4F80810E94261508950F9359
:102D00001F93CF93DF93082FC7E7D2E011E007C0EE
:102D100088810E945E151F5F2196193069F0101797
:102D2000B9F7E12FF0E0EA58FD4F80810E942615A7
:102D30001F5F2196193099F7DF91CF911F910F9165
:102D40000895E82F8150883008F00895F0E0EA589F
:102D5000FD4F80810E945E150895E82F81508830D4
:102D600008F00895F0E0EA58FD4F80810E94421576
:102D70000895E82F8150883010F080E00895F0E049
:102D8000EA58FD4F80810E94A8150895E82F8150D0
:102D9000883010F080E00895F0E0EA58FD4F80811F
:102DA0000E94C1150895CF93DF93C7E7D2E08991C0
:102DB0000E945E1582E0CF37D807C9F7DF91CF9127
:102DC00008958D3008F00895E82FF0E0E956FD4FA2
:102DD00080810E94261508958D3008F00895E82F0F
:102DE000F0E0E956FD4F80810E945E1508958D3018
:102DF00008F00895E82FF0E0E956FD4F80810E9429
:102E000042150895E7E9F2E0E80FF11D80810E9484
:102E1000A8150895CF93DF93C7E9D2E089910E9466
:102E20005E1582E0C43AD807C9F7DF91CF910895C3
:102E30000E940A1784E00E945E1583E00E945E15DE
:102E400088E00E945E1581E00E945E1582E00E948B
:102E50005E150895F894179820E030E0909158049A
:102E6000F901ED5AFB4F80819823F901E25BFB4F9A
:102E70008081982B9EBD0DB407FEFDCF2F5F3F4F85
:102E80002530310559F7179A78940895EEE4F4E067
:102E9000A3E5B4E080819D91892B819384E0E335A3
:102EA000F807C1F70895EEE4F4E0A3E5B4E09D91DE
:102EB000909580818923819384E0E335F807B9F701
:102EC0000895EEE4F4E0A3E5B4E020819C91892F1D
:102ED000822319F09095922390831D92319684E07D
:102EE000E335F80791F708951F93182F84E00E94A7
:102EF0005E15123049F083E00E945E15113071F0CA
:102F00001F3F39F01F91089583E00E9442151F91E1
:102F1000089584E00E9426151F91089583E00E9481
:102F200026151F9108950F931F93CF93DF93182FAA
:102F300087FD50C086E10E945A16812F82958695A2
:102F40008695837080FF29C085E10E9444161F7317
:102F500049F11731A0F58FEF0E94741784E10E94A8
:102F60005A16012F10E0CBE0D0E0C017D10731F0A6
:102F7000FE01E457FD4F80810E945E152196C83105
:102F8000D10599F704571D4FF80180810E9426153D
:102F9000DF91CF911F910F91089585E10E945A16FC
:102FA0001F73B9F680E00E9474170E940A1784E12B
:102FB0000E944416DF91CF911F910F910895143212
:102FC00068F0103370F4185181E00E9474171123D7
:102FD00029F6EBCF86E10E944416AFCF1C5080E06B
:102FE000F4CF1C3318F4145282E0EFCF105383E077
:102FF000ECCFEFE7F2E0E80FF11D80810E9426158B
:103000000895EFE7F2E0E80FF11D80810E945E1560
:103010000895E7E7F2E0E80FF11D80810E94261590
:103020000895E7E7F2E0E80FF11D80810E945E1548
:103030000895DF92EF92FF920F931F93CF93DF9348
:10304000F02EDE2C222371F1022F040FE42EC7E7AD
:10305000D2E010E00BC0101758F41F15D9F088818A
:103060000E9426151F5F2196183049F01E1598F70B
:1030700088810E945E151F5F21961830B9F781E0A4
:103080008D15A0F4DF91CF911F910F91FF90EF90DC
:10309000DF900895E12FF0E0E958FD4F80810E9414
:1030A0004215E0CF062F080FE82ED1CFDD2071F0BA
:1030B00088E00E945E1581E00E942615DF91CF9185
:1030C0001F910F91FF90EF90DF90089588E00E948C
:1030D000261581E00E945E15DF91CF911F910F911F
:1030E000FF90EF90DF900895FF920F931F93082FAA
:1030F000F62E84E00E945E1583E00E945E1588E053
:103100000E945E1581E00E945E15102F04FD34C000
:1031100015FD29C007FD2CC016FD21C00E940A170D
:10312000FF2099F0802F8F708D3098F08BE10E94F6
:1031300026158CE10E9426158FE00E9426158EE050
:103140000E9426158DE00E9426151F910F91FF9079
:1031500008950E94E1161F910F91FF90089581E05C
:103160000E942615DBCF83E00E94261507FFD4CFEF
:1031700088E00E942615D0CF84E00E942615C8CF93
:10318000E5E4F2E0E80FF11D808108958A3008F04F
:103190000895E82FF0E0E359FD4F80810E94261545
:1031A0000895CF93DF93CDE6D2E089910E945E151A
:1031B00082E0C737D807C9F7DF91CF910895909182
:1031C0004E04982790934E0490914F049827909323
:1031D0004F0490915004982790935004909151047B
:1031E00098279093510490915204982790935204F9
:1031F0000895AC0161157105A1F020E0E0E0A0E0C8
:10320000B0E0A40FB51F8C91E827F0E0E454FD4F27
:10321000E0812F5FA22FB0E0A617B70790F38E2FA3
:103220000895E0E0FCCF0E9479140E947E28882354
:10323000D1F30895EF92FF920F931F93CF93DF93F3
:103240007C018B016115710561F0C0E0D0E0F701F0
:10325000EC0FFD1F80810E94CE012196C017D1077F
:10326000B0F3DF91CF911F910F91FF90EF900895F0
:1032700022E42093E1041092E20422E02093E3048C
:103280009093E4048093E504A1EEB4E0E0E08D9136
:10329000E827F0E0E454FD4FE08184E0A63EB80763
:1032A000B1F7EC93CD01059766E070E00E941A1922
:1032B000089590E89093E1041092E20421E02093B5
:1032C000E3048093E404ACEBB2E090913C03FD0195
:1032D000E90FF11D90819227FD01E90FF11D908109
:1032E0009827A90FB11D8C918093E50481EE94E09D
:1032F00065E070E00E941A1908951F920F920FB6B0
:103300000F920BB60F921124DF92EF92FF920F9360
:103310001F932F933F934F935F936F937F938F935D
:103320009F93AF93BF93CF93DF93EF93FF9310914E
:10333000CE008091BB02882309F46EC080915B04AB
:1033400090915C04895E934008F080C0809159049C
:10335000803408F089C0282F2F5FE82FF0E0EF5D60
:10336000FA4F10832093590410925C0410925B046E
:10337000233008F451C0709121059091220580E01E
:1033800060912305462F50E0482B592B30E0CA01AD
:1033900004962817390708F43FC09A012D5F3F4F64
:1033A000F901EF5DFA4F10812115310509F401C1D2
:1033B00090E0E0E0A0E0B0E0AF5DBA4F8C91E8278C
:1033C000F0E0E454FD4FE0819F5FA92FB0E0A21729
:1033D000B30790F31E1709F450C02115310509F405
:1033E000EAC090E0E0E0A0E0B0E0AF5DBA4F8C91C1
:1033F000E827F0E0E454FD4FE0819F5FA92FB0E0A3
:10340000A217B30790F38E2F90E00E94AA011092AA
:10341000590480E00E945919FF91EF91DF91CF91FB
:10342000BF91AF919F918F917F916F915F914F91DC
:103430003F912F911F910F91FF90EF90DF900F9090
:103440000BBE0F900FBE0F901F9018950E94EA15AB
:103450000E942A171093210581E08093590410924D
:103460005C0410925B04D8CF0E9459191092590441
:1034700010925C0410925B04CFCF713809F492C1B2
:103480007238B0F5713109F42BC1723108F096C071
:10349000713051F1703131F080E00E945919109271
:1034A0005904BACF6231C1F780912405082F10E08A
:1034B000000F111F000F111F000F111F8091250514
:1034C000080F111D02951295107F1027007F1027FD
:1034D000C6E2D5E08991B8010E94701D0F5F1F4FB1
:1034E00085E0C633D807B1F781E00E945919D7CFDC
:1034F000763809F435C1773808F073C0723809F4AA
:1035000084C1753849F64330510509F0A5C03091A2
:103510002405932F80E020912505E22EFF24E82A40
:10352000F92AD0902605EAE3ED1508F4B6CF70939A
:10353000E1041092E204F2E0DF0ED092E3048EEF99
:10354000D80E3093E4042093E504DD2071F006EEFC
:1035500014E0E701CE010E94B41DF80181938F01B0
:1035600021969E012E192D15A8F38091E304682F52
:103570006D5F09F4D5C1A1EEB4E090E08E5F282F15
:1035800030E02E513B4F8D919827E92FF0E0E45425
:10359000FD4F9081A217B307B1F7E62FF0E0EF518E
:1035A000FB4F90836F5F81EE94E070E00E941A19E8
:1035B00076CFE0E00FCF80E090E027CF703409F4C1
:1035C00053C1713409F068CF623009F065CF909132
:1035D000240580E020912505820F911D0E94B402F0
:1035E0005ECF7738E9F1783809F056CF7093E1046F
:1035F0001092E20480912405813009F46AC181307F
:1036000008F05BC180E18093E4041092E5048093AC
:10361000E6041092E70484E047E0A7E0B0E068E049
:1036200070E08093E30490E020E030E0F901EF5196
:10363000FB4F80819827E92FF0E0E454FD4F908103
:103640002F5F3F4F241790F3AF51BB4F9C9381EEF8
:1036500094E00E941A1923CF80E00E9459191FCFCD
:1036600080912405882309F006C14230510509F0F4
:1036700014CFE0912505E43008F00ECF89E1809366
:10368000E1041092E20480E18093E3042E2F30E005
:1036900022953295307F3227207F3227A4EEB4E086
:1036A000F901E559F94F80818D932F5F3F4F84E0F9
:1036B000A43FB807A9F75397E0E08D91E827F0E021
:1036C000E454FD4FE081F4E0A43FBF07B1F7E0937D
:1036D000F404CD01439764E170E00E941A19DFCE33
:1036E000623009F0D9CE80912405082F10E0000F38
:1036F000111F000F111F000F111F80912505080FCA
:10370000111D02951295107F1027007F102789E167
:103710008093E1041092E20480E18093E304C4EE1C
:10372000D4E0C8010E94B41D89930F5F1F4F34E09D
:10373000C43FD307B1F7DE015397E0E08D91E8274E
:10374000F0E0E454FD4FE081CA17DB07B9F7E093DE
:10375000F40481EE94E064E170E00E941A199FCEB7
:103760009091240580E020912505E22EFF24E82A8F
:10377000F92A2EEFD22ED60E63506A3308F06CCFA2
:10378000DD2009F4B1CE06E215E0E701F8018191F0
:103790008F01BE010E94701D21969E012E192D15CC
:1037A000A8F3A2CE87E190E09093E5048093E4042F
:1037B0008BEC90E09093E7048093E604E4EBF2E076
:1037C000A8EEB4E081918D9322E0EA3BF207D1F7B5
:1037D00081E88093E1041092E2048AE08093E3049C
:1037E000A1EEB4E0E0E08D91E827F0E0E454FD4F75
:1037F000E08134E0AE3EB307B1F7EC93CD010D9715
:103800006EE070E00E941A194ACE4230510509F06C
:1038100023CF30912405332309F468C09091250506
:1038200020E082E88093E1041092E20483E0809338
:10383000E3043093E4049093E5042093E604A1EEBE
:10384000B4E0E0E08D91E827F0E0E454FD4FE08142
:1038500084E0A73EB807B1F7EC93CD01069767E087
:1038600070E00E941A191BCE80917C0490917D0417
:103870000E94381914CE813009F00ECE4231510524
:1038800009F00ACEE0912505E43008F005CE2E2F90
:1038900030E0A6E2B5E022953295307F3227207FD6
:1038A00032278D91F901E559F94F80832F5F3F4F02
:1038B00085E0A633B807A9F717CE883009F0ECCD1C
:1038C00081E08093E40444E0A4E0B0E065E070E0CF
:1038D000A8CE88E08093E40480E18093E50482E050
:1038E00045E0A5E0B0E066E070E09BCE9091250554
:1038F000973860F4953870F4993181F0993120F05F
:10390000892F8158823030F020E08BCF973821F01A
:103910009838D1F721E085CF24E083CF20E181CF13
:1039200090E03BCE2C98803408F08FE3611160E486
:10393000442349F090E0882349F0682B962B98B9EE
:103940002C9A2D9A089590E88823B9F7962B98B968
:103950000895882319F42D982C980895469A2C9848
:1039600008959F92AF92BF92CF92DF92EF92FF9213
:103970000F931F93CF93DF930E94EA1580919A04CF
:103980000E94F8150E9479140E944114BB249924C6
:10399000AA24CC240E9479140E947E28882309F04E
:1039A00073C02B2D3CE02302C001112497E1D92ED6
:1039B000D80EEA2CE294EE0CEE0C80ECE822C0E08B
:1039C000D0E009C0802F0E94E012882319F52196CB
:1039D000CD30D10559F1FC2EFE01E454FC4F00819D
:1039E000802F0E94CA12882369F31C2F1D0D812F7E
:1039F0006C2D4A2D0E94921C812F8E290E94BA0E96
:103A00008C2F0E94E116CC24C394802F0E94E012D8
:103A10008823E9F28F2D8D0D8E290E94F90E8F2DAE
:103A20000E94EC162196CD30D105A9F68FE00E94B8
:103A3000CA12882309F442C081E08B150CF04EC0F5
:103A40009B1429F08B2D0E9474170E942A1784E181
:103A50000E94CA12882351F080E0AA2009F481E074
:103A6000A82E8823B9F188E00E94261586B190E03F
:103A70008F739070892BB1F49B2C0E9479140E9453
:103A80007E28882309F48DCF0E94700FDF91CF919B
:103A90001F910F91FF90EF90DF90CF90BF90AF906C
:103AA0009F9008950E94F612882331F380E00E94CF
:103AB000A91C0E940A17CC249B2CDFCF8EE00E9409
:103AC000CA12882309F4BCCF2FEFB21609F4B8CF7D
:103AD000BA94B6CF88E00E945E15C8CFB394B0CF39
:103AE000282FF89495E028980000000000000000BE
:103AF0009EBD0DB407FEFDCF0000000000000000D9
:103B00001EBC0DB407FEFDCF8EB5289A0000000044
:103B10000000000080FDE7CF28980000000086E04C
:103B20008EBD0DB407FEFDCF00000000289A0000F6
:103B300000000000000028980000000082E08EBD18
:103B40000DB407FEFDCF7EBD0DB407FEFDCF6EBDEB
:103B50000DB407FEFDCF2EBD0DB407FEFDCF000056
:103B60000000289A78940895382FF89425E0289832
:103B700000000000000000002EBD0DB407FEFDCFC8
:103B800000000000000000001EBC0DB407FEFDCFC9
:103B90008EB5289A000000000000000080FDE7CFED
:103BA00028980000000083E08EBD0DB407FEFDCF15
:103BB0009EBD0DB407FEFDCF3EBD0DB407FEFDCF8B
:103BC000000000001EBC0DB407FEFDCF8EB5289A84
:103BD00078940895892F8F7184FD806E0895EF92F7
:103BE000FF920F931F93FA01D90186958083862F48
:103BF00090E08F70907095958795959587959595A0
:103C000087958C93862F8770F801808362956F70FB
:103C1000F70160831F910F91FF90EF900895FC01D1
:103C200030E022953295307F3227207F3227208363
:103C30008081660F660F660F640F6F70862B80831E
:103C4000089580915D04882349F087FD0EC083E0CC
:103C50000E94261584E00E945E15089583E00E946C
:103C60005E1584E00E945E15089583E00E945E1553
:103C700084E00E9426150895962F803110F08FEF72
:103C80000895682F70E0660F771F6F5F734F892F5D
:103C90000E94701D80E008959B01803120F5682FFF
:103CA00070E0FB01EE0FFF1FE753FC4F8081918115
:103CB00028173907A0F0009749F08150660F771F49
:103CC0006050744F0E94701D80E0089580E0660F80
:103CD000771F6050744F0E94701D80E00895C901E5
:103CE000009759F7F3CF8FEF0895803198F470E083
:103CF0006050784F90E000249695879507949695AC
:103D000087950794982F802D680F791F8CE060307D
:103D1000780710F08FEF0895842F0E94701D80E0C7
:103D20000895EF92FF920F931F93CF93DF93C82FC5
:103D3000D0E0CC0FDD1FCC0FDD1FCC0FDD1FC60F79
:103D4000D11DC05CDF4FCC0FDD1FC295D295D07F57
:103D5000DC27C07FDC27EE24FF248701000F111F22
:103D60000F591A4FF80180819181892FBE010E945D
:103D7000701DF801808191812196BE010E94701D05
:103D80000894E11CF11C2196F0E1EF16F10429F7EB
:103D9000DF91CF911F910F91FF90EF90089590E0E8
:103DA000880F991F8F5F934F0E94B41D90E0089574
:103DB0000F931F93082F10E0000F111FC8018050B0
:103DC000944F0E94B41D90E0019607531C4FF801D8
:103DD000208131818217930708F49C01C9011F914A
:103DE0000F9108958091D00480939205809192055F
:103DF0000E94D81E90938D0580938C05809192052A
:103E00000E94CF1E90939405809393052091930573
:103E10003091940580918C0590918D052817390774
:103E200020F0109294051092930580918105909155
:103E30008205E0919205F0E0EE0FFF1FE753FC4F83
:103E4000608171810E94AD459093820580938105C8
:103E50000895803198F470E06050784F90E000242D
:103E6000969587950794969587950794982F802D1A
:103E7000680F791F8CE06030780710F08FEF08959D
:103E8000CB010E94B41D0895EF92FF920F931F93F0
:103E9000CF93DF93E0908105F09082050894E11CB8
:103EA000F11C80E00E9409138823C9F400E080918E
:103EB0009505813029F180E00E94E012882329F0E5
:103EC00080919505882309F0BFC0013009F4E7C04F
:103ED000DF91CF911F910F91FF90EF90089581E0B6
:103EE000809395051092910510929005809364043B
:103EF00082E20E945E1501E0809195058130D9F63D
:103F00000E942714282F8823B9F021508091900512
:103F1000909191057C01EE0CFF1CEE0CFF1CEE0C49
:103F2000FF1C880F991FE80EF91EE20EF11CF0929B
:103F30009105E092900501E087E10E94CA12882372
:103F400041F0E0909305F09094050894E11CF11C79
:103F500001E083E00E94CA12882329F0E0908C05DA
:103F6000F0908D0501E089E00E94CA12882309F0D3
:103F7000A2C089E00E94E012882309F0BAC08AE05A
:103F80000E94CA12882309F0A5C08AE00E94E012AC
:103F9000882309F490CF8CE10E945E15E091920590
:103FA00020918C0530918D05F0E0EE0FFF1FE75357
:103FB000FC4F808191812817390708F07CCF8091D0
:103FC0008C0590918D05019690938D0580938C05BD
:103FD0008091920560918C0570918D050E944C1E18
:103FE000809192050E94D81E90938D0580938C0538
:103FF00060918C0570918D056150704080918105B4
:104000009091820586179707D8F4EB01219701C09C
:10401000E901809192051C2F6C2F0E94291F482FC7
:10402000809192051F5F612F0E94751E9E01215095
:10403000304080918105909182058C179D0740F357
:1040400088E08093670437CF82E20E9426151092A1
:1040500064041092950581E0809367042091900597
:104060003091910521153105A9F0E0919205F0E01C
:10407000EE0FFF1FE753FC4F80819181821793075A
:1040800048F021503040309382052093810587E02D
:104090008093670410923804013009F019CFC701EA
:1040A0000E94EB0100933804DF91CF911F910F9193
:1040B000FF90EF9008958BE10E94261510929105D4
:1040C00010929005E0908105F09082050894E11C23
:1040D000F11C4FCF8CE10E94261510929105109291
:1040E0009005E0908105F09082050894E11CF11C98
:1040F0004CCF8BE10E945E15C0918105D091820565
:10410000219680918C0590918D05C817D90708F0EC
:1041100036CF809192051C2F6C2F0E94291F482FAB
:10412000809192051150612F0E94751E21968091F9
:104130008C0590918D05C817D90758F380918C058F
:1041400090918D05019790938D0580938C058091BA
:10415000920560918C0570918D050E944C1E809196
:1041600092050E94D81E90938D0580938C0588E05F
:104170008093670404CFEF92FF920F931F93809177
:10418000D00480939205809192050E94D81E90934E
:104190008D0580938C05809192050E94CF1E90938F
:1041A0009405809393052091930530919405809117
:1041B0008C0590918D052817390720F010929405F1
:1041C000109293058091810590918205E09192056E
:1041D000F0E0EE0FFF1FE753FC4F608171810E94FA
:1041E000AD45909382058093810580919205609101
:1041F0008105709182050E94291F80938905809115
:1042000092056091890540EE55E028E935E00AE91C
:1042100015E0ECEAEE2EE6E0FE2E0E94EF1D81E0B6
:10422000809328060E94AF288091AC068093B30645
:104230001F910F91FF90EF900895AF92BF92CF9290
:10424000DF92EF92FF920F931F93CF93DF93C82ECD
:10425000DD24CC0CDD1CCC0CDD1CCC0CDD1CC60E16
:10426000D11C80E490E0C80ED91ECC0CDD1CC29499
:10427000D29410EFD122DC24C122DC24AA24BB2456
:10428000C6010E94B41DD82FC0E07501EE0CFF1CC2
:10429000E1E6F5E0EE0EFF1EF701D183C083008159
:1042A0001181C60101960E94B41D90E0082B192BC4
:1042B000F701118300830894A11CB11C82E090E0F7
:1042C000C80ED91E90E1A916B104D1F6DF91CF91A5
:1042D0001F910F91FF90EF90DF90CF90BF90AF9024
:1042E000089510928B0584E20E945E150E94D515F8
:1042F0000E9461171092260680E00E94A91C089572
:1043000010928A05109226061092830580E00E9482
:10431000A91C0E94D5150E9461170E94411408959E
:104320008091870590918805682F6770969587958D
:1043300096958795969587958F700E94842C6091AD
:104340008705709188059B0140E050E0DA01C901C2
:1043500080709078A070B070892F9A2FAB2FBB27F8
:1043600080936E04DA01C90180709074A070B070FF
:10437000892F9A2FAB2FBB2780936C04207030724B
:1043800040705070232F342F452F552720936D04F4
:1043900010929B05872F8F7184FD806E089581E0B8
:1043A00080938A0581E20E94261510926C04809108
:1043B0006C0480936D0480916D0480936E04109260
:1043C0008305109226068091610590916205909375
:1043D0008805809387058F5F9F4F89F010928F0526
:1043E00010929B0510927A040E94902180935D04A4
:1043F00080912F0480FDFCCF81E0809383050E9493
:10440000EA15089581E080938B0584E20E942615C9
:104410000E94EA150895DF92EF92FF920F931F9387
:1044200080911207882309F483C284E00E94332913
:1044300010928605809186058093850510929505DA
:1044400010929105109290050E94BB208091C406A5
:104450006091050740912106209127060BE616E0A2
:104460000E94C22B809121066091270640919A05F7
:104470002091280600919E05E09098050E94191849
:1044800057E0D52E07C0113009F4FBC00E94592B0C
:104490008823C9F00E9479141091AB061330D9F02B
:1044A000143088F31430D9F11D3081F781E00E9477
:1044B00039308091AB068D3049F3109272040E941E
:1044C000592B882339F70E94282B0E9479141091C8
:1044D000AB06133029F70E943929882309F09EC1C1
:1044E0000E94AB2A882321F0109264041092720477
:1044F0000E945F13882351F2182F11500E940A174F
:10450000812F0E94E1161093AC0680911207882338
:1045100009F0BCCF8091AC068093B306B7CF0E9460
:104520003929882309F05CC180919505882309F415
:104530004AC10E94441F83E00E940913882309F0A6
:104540003BC187E10E940913882309F02EC186E14F
:104550000E940913882309F468C0809128068823E3
:1045600009F0B0C18091AC068093B306E09081055C
:10457000F090820580918605882309F090C1809192
:104580002706882309F44AC010E0209105073091DE
:1045900021068091B30690E082959295907F9827AE
:1045A000807F98278093890580918905220F220FAB
:1045B000220F230F210F2F70282B20938905809124
:1045C00092056091810570918205409189050E9454
:1045D000751E1F5F809181059091820501969093D1
:1045E0008205809381050894E11CF11C809181056E
:1045F00090918205E0919205F0E0EE0FFF1FE753E6
:10460000FC4F608171810E94AD459093820580933B
:10461000810580912706181708F4B7CF809185058A
:10462000882309F052C1D0926704809167048730D3
:1046300009F407C180916704883009F459C1809159
:104640006704813009F4AEC08091AB06843011F06C
:104650001092720480911207882309F4DBC08091C4
:104660007104813009F012CF109271040E947E28EB
:10467000882309F40BCF1F910F91FF90EF90DF90EB
:1046800008950E943929882309F073C00E94441FAD
:1046900083E00E940913882339F583E00E94E01229
:1046A0008823F1F4909192058091D004981711F02D
:1046B0000E94BB208091AB06813011F010927204F1
:1046C00080911207882309F0B8C00E947E288823B1
:1046D00009F4DCCE1F910F91FF90EF90DF900895C9
:1046E00083E20E945E15DECF109282051092810552
:1046F0008091920560918105709182050E94291F29
:1047000080938905809192056091890540EE55E07E
:1047100028E935E00AE915E0ACEAEA2EA6E0FA2E2F
:104720000E94EF1D81E0809328068091AC06809363
:10473000B3060E94AF288091C4066091050740919E
:104740002106209127060BE616E00E94C22B8091DD
:1047500021066091270640919A0520912806009134
:104760009E05E09098050E94191883E20E94261584
:1047700094CF0E94D51582E20E94261510937204F0
:1047800081E20E945E15809121066091270640918A
:104790009A052091280600912106E09098050E9434
:1047A000191874CF109267044FCF81E0809386056B
:1047B00080E00E944215CBCE81E08093850583E2A4
:1047C0000E944215BECE0E94462B9091920596956E
:1047D0009093DA04882309F0ACCE0E943930A9CE38
:1047E0000E94D51582E20E94261581E08093720412
:1047F00081E20E9426158091210660912706409152
:104800009A052091280600912106E09098050E94C3
:1048100019188ACE81E00E94332921CF0E94D51534
:1048200011E01093640484E20E9426158091AC0686
:104830000E94E1161093720453CE84E00E94332943
:1048400044CF8091920560918105709182050E940C
:10485000291F80938905809192056091890540EE1A
:1048600055E028E935E00AE915E09CEAE92E96E0F2
:10487000F92E0E94EF1D11E0109328068091210669
:104880006091270640919A052091280600919E0587
:10489000E09098050E94191810936704D0CE1092EA
:1048A0008605809192056E2D0E943C1E8091920596
:1048B0000E94CF1E909394058093930580E00E9400
:1048C0005E155DCE0E94AF284DCE10928505809179
:1048D0009205B7010E944C1E809192050E94D81E3D
:1048E00090938D0580938C0583E20E945E159BCE8C
:1048F0008091920560918105709182050E94291F27
:1049000080938905809192056091890540EE55E07C
:1049100028E935E00AE915E0BCEAEB2EB6E0FB2E0B
:104920000E94EF1D81E0809328061092670487CED5
:1049300081E00E9433297CCDEF92FF920F931F9369
:1049400080911207882309F4AAC184E00E943329C8
:1049500010928605809186058093850510929505B5
:1049600010929105109290050E94BB208091C40680
:104970006091050740912106209127060BE616E07D
:104980000E94C22B809121066091270640919A05D2
:104990002091280600919E05E09098050E94191824
:1049A00008C0143009F45FC00E94592B882309F411
:1049B00090C00E9479141091AB06113091F70E94BB
:1049C0003929882309F0DAC083E00E94091388237B
:1049D00009F0F5C083E00E94E012882309F039C194
:1049E00080E00E940913882309F03CC180E00E9406
:1049F000E012882309F04BC1909192058091D00478
:104A00009817E1F00E94BB208091C40660910507D1
:104A100040912106209127060BE616E00E94C22B4A
:104A2000809121066091270640919A0520912806E1
:104A300000919E05E09098050E9419188091AB06A0
:104A4000813011F01092720480911207882309F0CE
:104A500043C00E947E28882309F4A6CF1F910F919E
:104A6000FF90EF9008950E943929882309F065C0CE
:104A700086E10E940913882309F053C083E00E9455
:104A80000913882309F041C080E00E94091388239C
:104A900039F580E00E94E012882379F58091AB0619
:104AA000843011F01092720480911207882309F467
:104AB00061C080917104813009F076CF1092710449
:104AC0000E947E28882351F60E94592B882309F0E2
:104AD00070CF0E94282B6DCF84E00E943329B9CF7C
:104AE00011E01093950582E20E945E151093380440
:104AF00080E00E94E012882389F282E20E9426155B
:104B00001092950510923804C9CF81E080938505F5
:104B100083E20E9426151092860580E00E945E15B1
:104B2000B3CF81E08093860580E00E942615109225
:104B3000850583E20E945E15A1CF0E94D51582E211
:104B40000E94261581E08093720481E20E9426155E
:104B5000809121066091270640919A0520912806B0
:104B600000912106E09098050E94191881E00E94AA
:104B700027027ECF81E00E9433299BCF0E94D5156A
:104B800082E20E9426151093720481E20E945E1553
:104B9000809121066091270640919A052091280670
:104BA00000912106E09098050E94191881E00E946A
:104BB000270283E00E940913882309F40BCF109287
:104BC0008205109281058091920560918105709116
:104BD00082050E94291F809389058091920560912A
:104BE000890540EE55E028E935E00AE915E07CEA60
:104BF000E72E76E0F72E0E94EF1D81E080932806D5
:104C00008091AC068093B3060E94AF288091C406C1
:104C10006091050740912106209127060BE616E0DA
:104C20000E94C22B809121066091270640919A052F
:104C30002091280600919E05E09098050E94191881
:104C400083E20E94261583E00E94E012882309F483
:104C5000C7CE83E20E945E1580E00E94091388237C
:104C600009F4C4CE11E01093950582E20E945E150E
:104C7000809181059091820501960E94EB0110932D
:104C8000380480E00E94E012882309F4B5CE82E265
:104C90000E9426151092950510923804ADCE81E041
:104CA0000E94332955CEEF920F931F9310925F0409
:104CB00080911207882309F41DC284E00E943329E1
:104CC0001092860580918605809385051092950542
:104CD00010929105109290050E94F21E07C01130AB
:104CE00009F48FC00E94592B8823C9F00E947914BF
:104CF0001091AB061330D9F0143088F31430D9F189
:104D00001D3081F781E00E9439308091AB068D30F3
:104D100049F3109272040E94592B882339F70E949C
:104D2000282B0E9479141091AB06133029F70E94AA
:104D30003929882309F0B0C00E94AB2A882321F0CA
:104D400010926404109272040E945F13882351F23F
:104D5000182F11500E940A17812F0E94E1161093FC
:104D6000AC0680911207882309F0BCCF8091AC0675
:104D70008093B306B7CF0E943929882309F0D5C0A4
:104D800080919505882309F4C3C083E00E9409132C
:104D9000882329F080915F04813009F487C187E17D
:104DA0000E940913882309F08CC080E00E94091337
:104DB000882309F092C080E00E94E012882309F065
:104DC0009AC08091AB06843011F0109272048091E9
:104DD0001207882309F46FC080917104813009F0B3
:104DE00081CF1092710480915F04882309F07ACFFB
:104DF0000E947E28882309F475CF1F910F91EF90B0
:104E000008950E943929882309F0D9C08091950519
:104E1000882309F4F9C083E00E940913882379F0FC
:104E200081E080935F0480915F04882309F432C19C
:104E300083E20E942615109282051092810580E07F
:104E40000E940913882309F0ECC0109195051130D8
:104E500009F4FFC080E00E94E012882309F089C0B5
:104E6000909192058091D004981711F00E94F21E43
:104E70008091AB06813011F010927204809112077C
:104E8000882309F4B5CF84E00E9433290E947E284C
:104E9000882309F427CFB1CF0E94D51511E01093D4
:104EA000640484E20E9426158091AC060E94E116FB
:104EB0001093720441CF81E00E94332910925F0465
:104EC0008BCF81E08093860580E00E94421580E0D0
:104ED0000E940913882309F46ECF11E01093950501
:104EE00082E20E945E151093380480E00E94E01276
:104EF000882309F466CF82E20E9426151092950558
:104F000080913804813009F4E6C01092380459CFFA
:104F10000E94462B9091920596959093DA048823EF
:104F200009F033CF0E94393030CF0E94D51582E28C
:104F30000E94261581E08093720481E20E9426156A
:104F4000809121066091270640919A0520912806BC
:104F500000912106E09098050E94191880915F0445
:104F6000882309F49BC083E20E9442150E942A17FD
:104F700007CF82E20E942615109295052091900598
:104F8000309191052115310591F0E0919205F0E005
:104F9000EE0FFF1FE753FC4F80819181821793072B
:104FA00030F021503040309382052093810580916C
:104FB0003804813009F480C01092380451CF0E9427
:104FC000D51582E20E9426151093720481E20E9498
:104FD0005E15809121066091270640919A052091E7
:104FE000280600912106E09098050E9419188091EA
:104FF0005F04882309F456C083E20E94261580913D
:105000009505882309F007CF0E94462B90919205C1
:1050100096959093DA04882309F0FDCE0E943930EA
:10502000FACE11E01093950510929105109290051B
:1050300082E20E945E158091810590918205019621
:105040000E94EB011093380410919505113009F07E
:1050500001CF0E942714482F882309F4FBCE41502A
:105060002091900530919105C901880F991F880FF3
:10507000991F880F991F220F331F820F931F840FD0
:10508000911D90939105809390050E94EB011093E0
:105090003804E0CE83E20E945E15CDCE83E20E940A
:1050A0005E1564CF83E20E945E15B0CE80938505C5
:1050B00083E20E94261573CE809121066091270617
:1050C00040919A052091280600912106E0909805CC
:1050D0000E94191871CF8091210660912706409196
:1050E0009A052091280600912106E09098050E94DB
:1050F00019180BCF81E00E943329E2CD9091CF04A3
:105100008091D504891731F08091CF048093D50424
:1051100081E0089580E0089580912806882391F029
:105120008091E0058093C4068091980580930507DF
:1051300080919A0580932106809128068093270606
:105140001092280680912706882329F0809127064F
:1051500080932706089581E0809327060895809123
:10516000E0058093C406809198058093050780919F
:105170009A05809321068091280680932706109235
:1051800028060895833059F0843050F0843029F097
:105190008091AC068093B30608951092AC060895F2
:1051A0008230B0F70895FC0187858F708D30C1F093
:1051B00030E020E190E080818F708E3061F09F5F61
:1051C00031969217C0F3892F913118F48150832BB7
:1051D000089580E1FBCF9923B1F780E0832B0895F8
:1051E00030E12FE0E7CF1F93DF93CF930F92CDB73E
:1051F000DEB7162F0E94D328898389818F708F5F35
:105200008093EB0310939E05898184FD08C086E09E
:105210008093E9030F90CF91DF911F91089588E06B
:105220008093E9030F90CF91DF911F910895E82FAC
:10523000F0E0EF73F070E451FC4F808108954093EB
:105240009C056093DF058093AB0681E08093240684
:105250000895882339F08091DF058093AB0681E0C3
:105260008093240608958093AB0681E08093240602
:10527000089580912406882319F01092240681E075
:1052800008953F924F925F926F927F928F929F927A
:10529000AF92BF92CF92DF92EF92FF920F931F9344
:1052A000CF93DF93462E4A015901662309F4C4C007
:1052B0009C01E901DD2400E0FF241FEF6624772430
:1052C000B2E05B2E33243394CE010E94D328F30145
:1052D000E155F94F8083C0802FE0C222C39440E0A3
:1052E00050E012C01E251F7BF1F4F501E00FF11D07
:1052F0003082FF2009F070C0DD24D3940F5F4F5F30
:105300005F4F1E2D4C1588F5642FFE01E40FF51F2D
:10531000E0802E2D30E0C9018F7090700F9709F456
:1053200055C0DD20F9F6F501E00FF11D5082EF2D9B
:10533000F0E0D401AE0FBF1FEC926295607FE75D95
:10534000F94F6083F3940024220F331F001C220FB7
:10535000331F001C232F302DDD24D394D2220F5F66
:105360004F5F5F4F1E2D4C1578F20894611C711C25
:105370006096641408F4A8CF003408F061C08F2D43
:10538000F501E00FF11D10820F5F0034C8F39FE3B9
:105390009F1550F09FEFEF2DF0E0E75DF94F908300
:1053A000F3942FE32F15B8F7DF91CF911F910F9151
:1053B000FF90EF90DF90CF90BF90AF909F908F9035
:1053C0007F906F905F904F903F900895F501E00FB0
:1053D000F11D1082DD2492CFEF2DF0E03197E80D22
:1053E000F91DE082FA94EF2DF0E0F394E75DF94FB8
:1053F000A081AF70BA2FBF5F808182958F70682FB8
:1054000070E0CB018B0F911D40970CF0BA2F002458
:10541000220F331F001C220F331F001C232F302D9F
:10542000DD24D394D22262957295707F7627607FB7
:105430007627B62BB08362CF00E0FF2480E0A0CFB8
:105440008F2DA5CF2F923F924F925F926F927F92B6
:105450008F929F92AF92BF92CF92DF92EF92FF9284
:105460000F931F93CF93DF935C01562E3A0169018E
:10547000662309F45DC0482EEC0130E060E0EE24C4
:10548000FF24FA9480E000E010E05FE04EE0342E6C
:105490002DE0222E9FEA892E96E0992E800E911EF5
:1054A000F40170817F707F5FDE0190E0442D4195B3
:1054B0000BC05C93223089F0E42EEA0E3F5F9F5FC1
:1054C0001196822F9717D0F4F601E30FF11D20817A
:1054D000213079F7882349F45C93F301E60FF11D3D
:1054E000F0806F5FFC9222E0E7CF5C93F501EE0D58
:1054F000F11D808180648083FC92DECF903158F46E
:10550000FE01E90FF11D30829F5F05C0FE01E90F2A
:10551000F11D50839F5F9031C8F3F401808184FDB9
:105520002F860F5F1F4F6096822F051508F4B2CFAC
:10553000DF91CF911F910F91FF90EF90DF90CF906F
:10554000BF90AF909F908F907F906F905F904F90A3
:105550003F902F90089580919C050E94E01288232F
:1055600039F08091DF058093AB0681E080932406BB
:10557000089510928B0584E20E945E1510926104DA
:1055800080E00E945E150E9461170E9465160E94CD
:10559000EA158091D9040E94F81580E00E94A91CA8
:1055A000089581E080938B0584E20E9426150E9475
:1055B000EA1580E00E94F81580E00E94A91C089579
:1055C000109226060E9465160E94EA150E94611735
:1055D0008091D9040E94F8151092220681E20E945F
:1055E0005E1580E00E94A91C109212078CEF0E94A9
:1055F000210F089510929B0581E08093220681E29D
:105600000E94261580E00E94A91C80912E04882308
:1056100021F480912F0480FDFCCF10922F04109272
:105620003E0410923D0410924304109245041092DF
:10563000440410928604809186048093880481E05B
:1056400080932606809312078AEF0E94210F089507
:1056500080917204882311F480E0089581E00E9413
:105660000913882321F081E080937304089581E079
:105670000E94CA12882381F380E00E94B41288231A
:1056800059F382E08093730481E0089588E00E94DA
:10569000B412882369F09091AB0688E080939C0552
:1056A0009093DF0583E08093AB0681E0809324062E
:1056B000089580912E04823011F080E008950E94B8
:1056C000500F8093070780E00895AF92BF92CF926A
:1056D000DF92EF92FF920F931F93CF93DF935B01C3
:1056E000C82EDD24C294D29450EFD522DC24C522EA
:1056F000DC24EE24C0E0D0E0FF24F39405C0219622
:10570000F394F1E1FF16B1F085010C0F1D1FC601E6
:105710008C0F9D1F0E94B41DF8018083EE2079F745
:1057200080818F708E3059F7EF2C2196F394F1E140
:10573000FF1651F7EE20A1F490E1F50187858F70F7
:105740008D30B9F0892F81508F70DF91CF911F91EB
:105750000F91FF90EF90DF90CF90BF90AF900895A2
:105760009E2D915051F791E0F50187858F708D3016
:1057700049F7903110F08EE1E8CF892F81508F707A
:105780008061E3CFBF92CF92DF92EF92FF920F93AF
:105790001F93CF93DF936801E82EFF24EE0CFF1CCC
:1057A000E60EF11CEE0CFF1CEE0CFF1CEE0CFF1CB9
:1057B000E40EF11CE294F29470EFF722FE24E7224B
:1057C000FE2430E022953295307F3227207F322729
:1057D000B22E222379F0C0E0D0E086010C0F1D1F0D
:1057E000C7018C0F9D1F0E94B41DF8018083219674
:1057F000CB1598F3DF91CF911F910F91FF90EF9010
:10580000DF90CF90BF900895EF92FF920F931F9378
:10581000CF93DF93182F062F0E942A17E12EFF2423
:10582000EE0CFF1CEE0CFF1CEE0CFF1CE00EF11C3E
:10583000E294F294A0EFFA22FE24EA22FE24C0E0D1
:10584000D0E0FE01EC54F94F8081BE016E0D7F1D4A
:105850000E94701D2196C031D10599F70E942A1728
:10586000DF91CF911F910F91FF90EF900895CF920C
:10587000DF92EF92FF920F931F93CF93DF93E22E6D
:105880006801082F10E0000F111F060F111D000FF7
:10589000111F000F111F000F111F040F111D029582
:1058A0001295107F1027007F1027FF24E294F294B6
:1058B00080EFF822FE24E822FE24FE2C82E00E94E3
:1058C00026150E942A17EE2089F0C0E0D0E0F601EC
:1058D000EC0FFD1F8081B8016C0F7D1F0E94701DB1
:1058E00084E00E94FB0D2196CF1588F382E00E9490
:1058F0005E150E942A17DF91CF911F910F91FF90A3
:10590000EF90DF90CF900895EF92FF920F931F9347
:10591000CF93DF93182F062F0E942A17E12EFF2422
:10592000EE0CFF1CEE0CFF1CEE0CFF1CE00EF11C3D
:10593000E294F29440EFF422FE24E422FE24C0E03C
:10594000D0E0CE018E0D9F1D0E94B41DFE01EC54CF
:10595000F94F80832196C031D10599F710926104E7
:1059600080E00E947B150E942A17DF91CF911F9142
:105970000F91FF90EF90089580912E04882349F4B1
:105980000E94A50080912E04813049F00E94691286
:1059900008950E94B00380912E048130B9F70E94CF
:1059A000701208959F92AF92BF92CF92DF92EF92C2
:1059B000FF920F931F9381E08093AB0680932406A0
:1059C00000E011E032E0F32E2FE0E22E94E0D92E39
:1059D00086E0C82EB7E0BB2EAAE0AA2EF0E29F2EEA
:1059E0000E9479148091AB06863009F46FC087302D
:1059F00008F0AAC0813009F456C1843089F780913B
:105A00002406882339F0109224061093670410921C
:105A1000650400E080919C050E94E012882331F12A
:105A20008091DF058093AB06109324060023E1F0FC
:105A300080916504882311F41093650480916504B6
:105A4000813210F09092650490910002809165047B
:105A5000981751F0809165048093000260910002D4
:105A600087E090E00E945002109238040E942714B0
:105A7000282F882381F0809165048A9DC00111241C
:105A800080936504809165048150820F8093650442
:105A9000F092670401E080916704882309F4A0CFA5
:105AA0009091000280916704823009F4FDC1892F32
:105AB00090E00E94EB0110933804109267040E945A
:105AC00079148091AB06863009F091CF809124063D
:105AD000882339F01092240610926704109265040E
:105AE00000E080919C050E94E012882349F080919B
:105AF000DF058093AB0610932406002309F0D7C17D
:105B000080916504882309F475C1209165042130D2
:105B100009F453C120916504223009F422C1809117
:105B20006704813009F43EC180916704823009F036
:105B300057CF109267040E94EA1580919A040E9440
:105B4000F8150E942A174CCF873009F450C08F30C7
:105B500009F046CF80912406882349F0109224064C
:105B6000109367048091D0048093660400E08091D4
:105B70009C050E94E012882349F08091DF05809304
:105B8000AB0610932406002309F068C10E94AD13F0
:105B9000882369F0982F9150933048F480919404B1
:105BA000981729F0909394041093670401E0809172
:105BB0009404813009F436C180916704882309F484
:105BC0000FCF109267040E94D3160E94EA158091AD
:105BD00094048F5F0E94731680919404813009F0C1
:105BE000FFCE8091970481500E94F815F9CE8091E4
:105BF0002406882321F010922406109367048091D4
:105C00009C050E94E012882351F08091DF0580936B
:105C1000AB06109324068091670481FD31C10E9478
:105C2000AD13882389F0982F9150933068F48091B8
:105C30002E04981749F090932E040E94BC2C80915A
:105C4000670483608093670483E00E94CA128823FC
:105C500079F080916A048F5F80936A0480916A046E
:105C6000817080936A0480916704836080936704E5
:105C70008091670480FFB4CE809167048E7F80930B
:105C800067040E94D31680912E048F5F0E947316C2
:105C900083E20E945E1580916A04882309F414C18E
:105CA0000E942A179DCE80912406882331F01092FD
:105CB00024060E94D5150E942A1787E10E94091325
:105CC000882359F09091AB0687E180939C059093CF
:105CD000DF05B092AB061093240688E00E940913FA
:105CE000882359F09091AB0688E080939C059093AF
:105CF000DF05C092AB061093240681E00E940913D1
:105D0000882351F08091AB0610939C058093DF05AA
:105D1000D092AB06109324068EE00E9409138823CC
:105D200059F09091AB068EE080939C059093DF052F
:105D3000E092AB06109324069091CF048091D50495
:105D4000891709F44DCE8091CF048093D5041F911B
:105D50000F91FF90EF90DF90CF90BF90AF909F900A
:105D600008959091D00480916604981759F080911D
:105D7000D004809366042093670480916604809326
:105D80009A0401E089E00E94E012882309F4C7CE5A
:105D9000109265048BE10E945E158091670481304A
:105DA00009F0C2CE109267040E94EA158091AD04FA
:105DB0000E94F8150E942A1713CE9091D00480916A
:105DC0006604981759F08091D0048093660420935C
:105DD0006704809166048093AD0401E08AE00E942C
:105DE000E012882309F496CE109265048CE10E949B
:105DF0005E1590CE8AE00E94CA12882309F068C01E
:105E000089E00E94CA12882309F47FCE8BE10E94A8
:105E10002615F0926504F09267048091D004809377
:105E2000660473CE909166048091D004981709F4AB
:105E3000C3CE8091D00480936604909166049F5FE6
:105E4000923008F451C080919704981709F4B4CEA9
:105E5000909397041093670401E0AECE809197046D
:105E60006091940490E0019782959295907F982795
:105E7000807F9827682B8AE090E00E94500286CEAF
:105E800080916A0490E08170907082959295907FE5
:105E90009827807F982760912E046F70682B82E08E
:105EA00090E00E945002BBCE9091650400CE83E04A
:105EB00090E06091AD040E94500284E090E0609117
:105EC0009A040E9450021CCE83E20E942615E8CE5E
:105ED0008CE10E942615109365041093670480914D
:105EE000D004809366048CCF92E0ADCF0F931F93C4
:105EF0008091AC068093B306809128068823C9F070
:105F00008091E0058093C4068091980580930507F1
:105F100080919A0580932106809128068093270618
:105F20001092280680916404823088F01F910F91AE
:105F3000089590910507809198059817B9F380917D
:105F40006404823098F780919805809305078091CA
:105F5000C4066091050740912106209127060BE6B3
:105F600016E00E94C22B609121068091AD069091AF
:105F7000AE060E94F3281F910F9108951092120708
:105F800080E00E94A91C8CEF0E94210F80912E04BA
:105F9000813011F00E943F1210926906109286041F
:105FA0008091860480938804109299058BE696E090
:105FB0009093AE068093AD068091D5048D3039F074
:105FC000833029F08B3019F0873009F008950E9452
:105FD000762F08951F93DF93CF930F92CDB7DEB73F
:105FE00080E00E94A91C1092690610922F04109262
:105FF0003E0410923D041092430410924504109206
:106000004404109274041092860480918604809354
:106010008804109299058BE696E09093AE068093E3
:10602000AD06109121060E94D328898389818F7043
:106030008F5F8093EB0310939E05898184FD17C0C9
:1060400086E08093E90383E0809312078AEF0E9441
:10605000210F80912E04813011F00E943D1283E0C7
:10606000809336040F90CF91DF911F91089588E0BF
:10607000E8CFEF920F931F93982F882309F495C0D0
:10608000813029F080E01F910F91EF900895809169
:106090002406882309F0F9C00E94AD13882399F1E2
:1060A000982F915080912806882341F480912106F1
:1060B00080939A058091C4068093E00580919A05AB
:1060C000891770F480919A05981B9F5F909328061A
:1060D00080912806853008F446C184E08093280624
:1060E00080911207882309F441C1809121066091B3
:1060F000270640919A052091280600919E05E09080
:1061000098050E94191884E10E94CA12882309F098
:10611000DEC085E10E94CA12882309F0CEC08091BA
:106120001207882321F5909105078091980598170B
:10613000F1F080919805809305078091C4066091E5
:10614000050740912106209127060BE616E00E94E4
:10615000C22B809121066091270640919A052091DB
:10616000280600919E05E09098050E9419188091DC
:106170001207882329F480912806882309F0D4C0C7
:106180000E94C713982F882309F47CCF809165045F
:106190009150981709F076CF8091DF058093AB0678
:1061A00081E08093240680E06ECF0E94AD13982F8B
:1061B0008823D1F584E10E94CA12882309F49FC084
:1061C0001092980588E00E94261581E00E945E15D5
:1061D00080911207882309F055CF9091050780918F
:1061E0009805981709F44ECF80919805809305077C
:1061F0008091C406609105074091210620912706F1
:106200000BE616E00E94C22B8091210660912706C2
:1062100040919A052091280600919E05E0909805EE
:106220000E94191880E02FCF8091DA048093E00556
:1062300001E000932806192F115010939A0584E16C
:106240000E94B412882309F44BC01092980588E08C
:106250000E94261581E00E945E15109365048091CE
:10626000AB068093DF058DE08093AB0681E08093E1
:1062700024061092AC0680911207882309F44FC0BF
:1062800081E01F910F91EF90089510922406909352
:106290007204809121066091270640919A05209111
:1062A000280600919E05E09098050E9419180E940A
:1062B000AD13882309F427CFF3CE81E080939805AE
:1062C00088E00E945E1581E00E94261528CF10927A
:1062D000980588E00E94261581E00E945E1519CF7E
:1062E00085E10E94B412882309F4B7CF0093980582
:1062F00088E00E945E1581E00E942615AECF85E100
:106300000E94CA12882309F463CF81E08093980524
:1063100088E00E945E1581E00E94261559CF82E038
:106320000E94C22881E0ADCF8091E0058093C40631
:10633000809198058093050780919A0580932106A6
:106340008091280680932706109228068091C40623
:106350006091050740912106209127060BE616E083
:106360000E94C22B0DCF80912806B8CE8091E00507
:106370008093C406809198058093050780919A05C3
:106380008093210680912806809327061092280684
:106390008091C4066091050740912106209127064F
:1063A0000BE616E00E94C22BA0CE2F923F924F9296
:1063B0005F926F927F928F929F92AF92BF92CF9295
:1063C000DF92EF92FF920F931F93DF93CF930F9281
:1063D000CDB7DEB70E9479141092AC068091AC065E
:1063E0008093B30680911207882311F40C94693BC3
:1063F00084E08093AB0681E0809324066624992490
:10640000882455247724739438E0432E26E0322ED6
:1064100093E0292E0E9479141091AB061830D9F020
:10642000193008F04CC0153009F49EC4163008F03D
:1064300096C0113009F431C2143009F40CC40E9422
:10644000592B882339F70E94282B0E947914109128
:10645000AB06183029F780912406882349F0109262
:1064600024060E94D51583E20E94261570926404CA
:1064700080919C050E94E0128823A1F08091DF05A5
:106480008093AB0670922406109264048091C40637
:106490006091050740912106209127060BE616E042
:1064A0000E94C22B0E94AD13882309F00FC50E94E1
:1064B000C713882321F281500E941118C0CF1B30CE
:1064C00009F4DEC21C30D0F5193009F485C21A3047
:1064D00009F0B5CF809124068823F9F010922406A4
:1064E00080E00E9426150E942A178091C4066091C0
:1064F000050740912106209127060BE616E00E9431
:10650000372C80E00E945E150E942A1784E0809359
:10651000AB0670922406109264048091670488236D
:1065200039F084E08093AB067092240610926704E1
:10653000809167048F5F8093670481CF1C3009F4DA
:106540007CC11D3009F07BCF81E00E943930809101
:10655000AB068D3009F473CF1092720470CF1630F1
:1065600009F4FCC0173009F06ACF80912406882313
:1065700089F1109224060E94D515609127068BE6BA
:1065800096E045EC56E02FE935E00E94412980E095
:106590000E9426151092670489E08093650410928A
:1065A000660480912706882391F020E0E22FF0E036
:1065B000E155F94F9081809166048F5F9F70890F3C
:1065C000809366042F5F80912706281778F366244E
:1065D0009924552480E00E940913882311F0662431
:1065E000639488E00E940913882311F012E0612E61
:1065F00087E10E940913882311F0B3E06B2E80918C
:106600006504893009F4E7C680916504813009F496
:10661000BCC680916504882309F491C58091650406
:10662000882329F080916504807F09F45FC0109170
:1066300065048EE00E94CA12882351F0809165049F
:1066400080618093650485E080936704F2E05F2EAB
:106650008FE00E94CA12882351F080916504806205
:106660008093650485E0809367045524539484E106
:106670000E94CA12882349F0809165048064809347
:10668000650485E08093670455248EE00E94E01243
:10669000882341F080916504807E8093650484E0C6
:1066A000809367048FE00E94E012882341F080917C
:1066B0006504807D8093650484E08093670484E1B1
:1066C0000E94E012882341F080916504807B8093D2
:1066D000650484E08093670480916704853009F441
:1066E0004EC580916704843009F460C580916504CB
:1066F000883009F43CC48091670490E08370907006
:10670000892B09F04CC4662009F499CE60912706C4
:106710008BE696E045EC56E02FE935E00E94222A10
:106720008091C406609105074091210620912706BB
:106730000BE616E00E94372C91E0691609F446C575
:10674000E2E06E1609F474C0F3E06F1609F077CE3C
:1067500087E08093AB067092240671CE8091240668
:106760008823D9F0109224060E94D515609127063F
:106770008BE696E045EC56E02FE935E00E94412992
:1067800084E20E9426151092670410926604E3E6E4
:10679000E093650466249924882480E00E9409130C
:1067A000882311F06624639488E00E9409138823EB
:1067B00011F082E0682E80916504833609F41EC5CD
:1067C00080916504813009F428C580916504833087
:1067D00009F486C580916504882309F451C4809129
:1067E000670490E083709070892B09F019C46620CB
:1067F00009F425CE609127068BE696E045EC56E03D
:106800002FE935E00E94222A8091C4066091050795
:1068100040912106209127060BE616E00E94372CB6
:1068200091E0691609F4D2C4E2E06E1609F007CED1
:106830003092AB067092240602CE80912406882303
:1068400089F010922406909162048091270698178F
:1068500009F42CC6709267048091DF058093AB0623
:106860007092240680919C050E94E012882309F40E
:10687000E6CD8091DF058093AB067092240680916F
:106880006704882309F4B7C58DE00E945E1582E095
:106890000E945E150E942A17D2CD8091240688237B
:1068A000E9F01092240680E00E9427020E94D5158C
:1068B00082E20E9426151093720481E20E945E1506
:1068C000809121066091270640919A052091280623
:1068D00000912106E09098050E94191880E00E941E
:1068E000393080E00E94CA12882329F085E0809325
:1068F000AB067092240683E00E94CA12882351F0EE
:106900008091AB0620929C058093DF054092AB06F8
:106910007092240688E00E940913882321F03092A7
:10692000AB067092240687E10E940913882329F0A0
:1069300087E08093AB06709224068BE00E940913D7
:10694000882359F09091AB068BE080939C0590933F
:10695000DF058093AB06709224068DE00E94091338
:10696000882361F09091AB068DE080939C05909315
:10697000DF059CE09093AB06709224068091AB06F5
:10698000813011F01092720480911207882329F04F
:1069900084E08093AB06709224069091CF0480919E
:1069A000D504891709F44BCD8091CF048093D50489
:1069B0000F90CF91DF911F910F91FF90EF90DF909B
:1069C000CF90BF90AF909F908F907F906F905F908F
:1069D0004F903F902F90089580912406882371F066
:1069E0001092240682E20E945E1581E00E94A91C9A
:1069F00080E00E94A91C80E00E942702909165041B
:106A000080919D059817C9F09090650480919D052F
:106A10008093650480916704833009F4AAC580914E
:106A20006704823050F080919705882331F4E0911B
:106A30006504F0E0E156FA4F708286E10E94CA12C6
:106A4000882329F080919705882309F450C5809107
:106A50006704833009F4BFC386E10E94E0128823F3
:106A600009F4EDCC80916704823009F0E8CC709293
:106A7000670480E00E94A91C82E00E945E15DFCCC2
:106A800080912406882361F01092240682E20E94FD
:106A90005E158FE00E9426150E942A171092670447
:106AA00080919C050E94E012882309F442C08091E5
:106AB000DF058093AB0670922406809167048823DB
:106AC00091F58091C406309105072091210690E050
:106AD000880F991F830F911D880F991F880F991F89
:106AE000880F991F280F20936304809127068093B5
:106AF00062048823C1F090E0A0E0B0E0282F30E0ED
:106B000022953295307F3227207F3227FD01E559CB
:106B1000F94F8081AF51BA4F8C939F5FA92FB0E09E
:106B2000A217B3079CF38FE00E945E158DE00E94D0
:106B30005E158DE00E94CA12882309F480CC8091F2
:106B40006704882309F07BCC80916204882309F4D0
:106B500076CC709267048091C4062091050710914D
:106B6000210690E0880F991F820F911D880F991FB1
:106B7000880F991F880F991F180F809163041817A9
:106B800009F45DCC8DE00E94261582E00E94261556
:106B90000E942A176091630480912706882309F4D4
:106BA00040C0C62EDD24C294D294A0EFDA22DC24A9
:106BB000CA22DC24A12EBB24A294B294F0EFBF22FF
:106BC000BA24AF22BA24750100E010E0C6010E9489
:106BD000B41D882E0559194FF8018083C7010E9402
:106BE000B41DB6010E94701D882DB7010E94701D52
:106BF00084E00E94FB0D0894C11CD11C0894E11C88
:106C0000F11C8E2D8A19082F10E08091270690E044
:106C100082959295907F9827807F9827081719076B
:106C2000ACF2109121068BE696E00E94D32889836E
:106C300089818F708F5F8093EB0310939E0589810C
:106C400084FD51C586E08093E90382E00E945E15D1
:106C50000E942A17F4CB809124068823E9F0109231
:106C600024060E94D51582E20E94261570927204B5
:106C700081E20E94261580912106609127064091AD
:106C80009A052091280600912106E09098050E941F
:106C9000191881E00E94270283E00E9409138823CB
:106CA00009F445C080912806882309F00DC490910D
:106CB000050780919805981781F080919805809339
:106CC00005078091C4066091050740912106209137
:106CD00027060BE616E00E94C22B609127068BE682
:106CE00096E045EC56E02FE935E00E94412980E02E
:106CF00090E0FC01E156FA4F108201968034910534
:106D0000C1F782E080936404109208071092660431
:106D100010926504109267041092970570926904AE
:106D200089E08093AB067092240699249A9480910E
:106D3000AB06843011F01092720480911207882300
:106D400021F47092AB067092240680917104813018
:106D500009F075CB109271049091CF048091D50405
:106D6000891709F021CE6BCB809124068823C9F0C6
:106D7000109224060E94D515709267048BE696E067
:106D80000E94D328282F2F702F5F2093650490E056
:106D9000929582958F7089279F7089278170809343
:106DA00066048EE00E944814823009F4D3C08AE061
:106DB0000E944814823009F4C4C089E00E9448143B
:106DC000823009F4B2C08FE00E94CA12882399F081
:106DD0002092670480916604882319F49CE09093C4
:106DE0006504809166048F5F8093660480916604D9
:106DF0008170809366048091670480FF21C0809138
:106E0000670481508093670480916604882309F4A5
:106E1000AAC180916504803108F4A8C381E0809301
:106E2000650483E00E94261580916504882309F09B
:106E300097C181E080936504809165040E940316E8
:106E400080E00E94E012882309F4F9CA8091670467
:106E50008230B8F182E0809364048BE696E061E0D2
:106E600045EC56E02FE935E00E94412990916504F8
:106E700080916604811180E191509F70892B8093ED
:106E8000AF068BE696E061E045EC56E02FE935E091
:106E90000E94222A8091C406609105074091210634
:106EA00021E00BE616E00E94372C8091C406609129
:106EB000050740912106209127060E94C22B1092BF
:106EC00064047092AB0670922406B9CA182F115050
:106ED000812F0E9409188091C40690910507E82E21
:106EE000FF24EE0CFF1CE90EF11CEE0CFF1CEE0C57
:106EF000FF1CEE0CFF1CE10EF11CE294F29450EF2B
:106F0000F522FE24E522FE248701005F1F4F8FE05B
:106F1000B7010E94701D84E00E94FB0D0894E11CE3
:106F2000F11CE016F10699F7C2CA8091650490E061
:106F30000E968F7090708F5F809365042092670427
:106F400042CF809165048F708F5F8093650420929B
:106F5000670433CF80916704823008F482C3809144
:106F600065048F5F809365042092670420CFE92D2C
:106F7000F0E0E156FA4F508293948091660498169F
:106F800010F06624639470926704109265048091F7
:106F9000670490E083709070892B09F4B4CB0E9451
:106FA000EA15809127068823B1F090E080E001C0C7
:106FB0008E2FE92FF0E0E155F94FE081EF70EF5FA0
:106FC000E80F981618F09E1608F4DCC29F5F8091B7
:106FD0002706981768F384E00E945E1583E00E94FC
:106FE0005E1588E00E945E158091670480FD13C0E5
:106FF000F2E05F1609F479C381E0581609F479C309
:10700000552031F084E00E94261583E00E94261569
:1070100088E00E9426150E942A171092670473CBFD
:107020000E94EA15E92DF0E0E75DF94F80818F3F7E
:10703000D1F0108112951F7000810F70010F0F5F4A
:10704000101738F010C0812F0E9421161F5F1017F3
:1070500050F48091670480FDF6CF812F0E94F815CF
:107060001F5F1017B0F38091670480FFBFC1882DA8
:1070700060E00E947418109267040E942A17B7CB30
:1070800086E10E94CA12882309F0B8C20E945F13E9
:10709000882309F081C287E10E94E012882329F049
:1070A0008FE3980E9822709267048EE00E94CA12B5
:1070B000882321F090E1892A709267048FE00E9472
:1070C000CA12882321F0E0E28E2A7092670484E1DC
:1070D0000E94CA12882321F0F0E88F2A7092670478
:1070E00085E10E94CA12882321F080E4882A7092E8
:1070F00067048EE00E94E012882321F09FEE89222F
:10710000709267048FE00E94E012882321F0EFED77
:107110008E227092670484E10E94E012882321F09D
:10712000FFE78F227092670485E10E94E0128823B6
:1071300009F455CB8FEB88227092670450CB86E11F
:107140000E940913882309F469CAE92DF0E0E15689
:10715000FA4F50807092650482E0809367045ECAA3
:107160008091650467CE80916504813108F4FBC18C
:1071700081E08093650483E00E945E1555CE112363
:1071800009F0E8C180916504882309F4E3C1662011
:1071900029F4E92DF0E0E156FA4F508282E0809325
:1071A000670480916704843009F0A0CA112359F064
:1071B00080916504882339F493948091660498162D
:1071C00010F0662463947092670490CA6092AB06D4
:1071D0006092240634C90E94F713882309F43CCC3A
:1071E00082E08093670486E10E94B412882309F04C
:1071F00033CC709267040E94A91C2ECC88E00E94B8
:10720000E012882309F4DCCA1092650470926704C6
:1072100080916504813009F0D8CA86E10E94E012AD
:10722000882309F023C28EE00E94CA12882349F005
:10723000882D80958071FFEE8F22882A82E08093CE
:1072400067048FE00E94CA12882349F0882D809538
:1072500080729FED8922882A82E08093670484E10E
:107260000E94CA12882349F0882D80958078EFE724
:107270008E22882A82E08093670485E10E94CA12E8
:10728000882349F0882D80958074FFEB8F22882A0F
:1072900082E0809367040E945F13182F882309F40B
:1072A00094CA80E00E94A91C85E00E94FB0D115049
:1072B0001F7080EF8822812AE82DF0E0EF73F070D4
:1072C000E451FC4F482D4078808160E00E94921C80
:1072D00082E08093670480916504833009F07ACA64
:1072E0000E945F13182F0E947913882319F4112329
:1072F00009F470CAE92DF0E0EB53F94F808280E089
:107300000E94A91C85E00E94FB0D93949FE39915B0
:1073100018F4109266049924709267041092650420
:10732000112309F457CA812E8A94EFE08E228EE051
:107330000E94B412882311F0F0E18F2A8FE00E949E
:10734000B412882311F080E2882A84E10E94B412EA
:10735000882311F090E8892A85E10E94B4128823DD
:1073600011F0E0E48E2AE82DF0E0EF73F070E451C4
:10737000FC4F482D4078808160E00E94921C82E0A2
:10738000809367042092650425CA86E10E94E0127A
:10739000882311F0409265048EE00E94CA1288236F
:1073A00029F082E080936704A2E05A2E8FE00E94C9
:1073B000CA12882329F082E08093670455245394ED
:1073C00084E10E94CA12882309F423C982E08093D1
:1073D000670455241EC987E10E94E012882309F43E
:1073E00013C910926504709267040EC9882D61E07C
:1073F0000E94741840CE82E00E9426150E942A172F
:107400009091C40620910507309121068091620475
:107410008823B9F1E92EFF24EE0CFF1CE20EF11CCB
:10742000EE0CFF1CEE0CFF1CEE0CFF1CE30EF11C1F
:10743000E294F29450EFF522FE24E522FE24870127
:10744000A0E0B0E0FD01EF51FA4F8081A559B94F9E
:107450008C93B8010E94701D84E00E94FB0D0F5FA9
:107460001F4F802F8E19A82FB0E08091620490E00A
:1074700082959295907F9827807F9827A817B907C3
:107480000CF3109121068BE696E00E94D3288983A5
:1074900089818F708F5F8093EB0310939E058981A4
:1074A00084FDE2C086E08093E903EEC9992309F4E4
:1074B000D1C982E20E945E158DE00E9426150E94CD
:1074C0002A1710926704CEC98091E0058093C40604
:1074D000809198058093050780919A0580932106F5
:1074E000809128068093270610922806EACB82E036
:1074F000809367040E94E113882311F020926704AF
:10750000E0916504F0E0E156FA4F82E08083E0917B
:107510006604F0E0EB53F94F808080922506E82D59
:10752000F0E0EF73F070E451FC4F482D407880811B
:1075300060E00E94921C80916504981639F090904A
:107540006504809166048F5F8093660482E00E94E8
:1075500026157DCA939480916604981608F417CE78
:10756000662463941BCE8091650403CE80916504EC
:1075700056CC0E94E113882309F051CA82E080931F
:1075800067044DCA992D981B8091670480FF9DC0A8
:10759000892F0E9421161FCD882E8A94FFE08F220A
:1075A0008EE00E94B412882311F080E1882A8FE0D7
:1075B0000E94B412882311F090E2892A84E10E948B
:1075C000B412882311F0E0E88E2A85E10E94B412FB
:1075D000882311F0F0E48F2AE82DF0E0EF73F070CB
:1075E000E451FC4F482D4078808160E00E94921C5D
:1075F00082E080936704209265044DCDE92DF0E090
:10760000EB53F94F80808EE00E94B412882311F072
:10761000F0E18F2A8FE00E94B412882311F080E2FB
:10762000882A84E10E94B412882311F090E8892A04
:1076300085E10E94B412882311F0E0E48E2AE82D3F
:10764000F0E0EF73F070E451FC4F482D40788081FA
:1076500060E00E94921C82E080936704709265044F
:1076600015CD109265047BCC88E01DCFE92DF0E0AC
:10767000EB53F94F80828EE00E94B412882381F58B
:1076800088248FE00E94B412882311F0F0E28F2A40
:1076900084E10E94B412882311F080E8882A85E1F1
:1076A0000E94B412882311F090E4892A80E00E949D
:1076B000A91C9394EFE3E91518F410926604992439
:1076C0007092670410926504AECD892F0E94F81560
:1076D00082CC81E08093AB06809324060C94FE312B
:1076E00000E1802ECECF88E0AECA84E00E9426154D
:1076F00092CC83E00E9426158ECC0F931F93CF93DC
:10770000DF93EC01442319F18B0150E070E020E09D
:1077100030E0F901E155F94F60816F706F5FD8017A
:1077200090E0FE01E50FF11D80818D939F5F5F5F0B
:107730009617B8F3760F2F5F3F4F005F1F4F241748
:1077400040F3872FDF91CF911F910F91089570E043
:10775000872FDF91CF911F910F910895BF92CF9204
:10776000DF92EF92FF920F931F93CF93DF936B0102
:10777000B42E442369F17C0110E000E0C0E0D0E0C9
:10778000C7010E94D328FE01E155F94F8083208173
:107790002F702F5FD70190E08D91F601E10FF11D61
:1077A00080839F5F1F5F9217B8F3020F219680E1DD
:1077B00090E0E80EF91ECB1518F3802FDF91CF91E2
:1077C0001F910F91FF90EF90DF90CF90BF900895A1
:1077D00000E0F3CFCF92DF92EF92FF920F931F93CF
:1077E000DF93CF93CDB7DEB7C054D0400FB6F89437
:1077F000DEBF0FBECDBF109267041092650482E019
:1078000080936404409127068BE696E06E0108940D
:10781000C11CD11CB6010E94AE3BE82E80916604CB
:107820008E1510F010926604809127068823C1F00F
:1078300090E030E0E32FF0E0E155F94F20812F7028
:107840002F5F80E0E92FF0E0E75DF94F80838F5FE5
:107850009F5F8217B8F33F5F80912706381750F378
:107860000E94791480911207882309F4C5C184E02D
:107870000E943329FF240E9479141091AB06113025
:1078800071F01430E1F10E94592B8823A1F70E9476
:10789000282B0E9479141091AB06113091F70E94A9
:1078A0003929882309F0F4C086E10E94091388234E
:1078B00029F080916804882309F088C18091AB0683
:1078C000813011F01092720480911207882309F020
:1078D00070C10E947E288823B1F210926404C05CBB
:1078E000DF4F0FB6F894DEBF0FBECDBFCF91DF9153
:1078F0001F910F91FF90EF90DF90CF9008950E941D
:107900003929882309F037C110E086E10E94091364
:10791000882309F0D0C087E10E940913882309F069
:10792000E6C086E10E94E012882309F0FCC087E1EE
:107930000E94E012882309F001C186E10E94CA1268
:10794000882309F006C18EE00E94CA12882339F00C
:107950008F2D809580719FEEF922F82A12E08FE03A
:107960000E94CA12882339F08F2D809580729FED76
:10797000F922F82A12E084E10E94CA12882339F021
:107980008F2D809580789FE7F922F82A12E085E113
:107990000E94CA12882339F08F2D809580749FEB46
:1079A000F922F82A12E00E945F13282F882361F041
:1079B0008F2D90E08F7090700D9734F421502F70C0
:1079C00080EFF822F22A12E088E00E94CA1288238F
:1079D00009F44AC08F2D90E08F7090700D970CF4D1
:1079E000ECC090EFF92200E010E080916604F6010F
:1079F000E80FF11DF08240912706C6016BE676E0A4
:107A00000E947D3BE82E81E0809368040D301105D3
:107A1000BCF58F2D61E00E94741884E20E94261547
:107A20000E94EA15E0916604F0E0E75DF94F80817D
:107A30000E94F8150E942A178091AB06843011F03D
:107A40001092720480911207882309F4AEC08091CD
:107A50007104813009F017CF109271040E947E28C2
:107A6000882309F410CF39CF123009F4C9C011307E
:107A700019F70F2D10E00F7010700D3011054CF23A
:107A80008F2D60E00E94741884E20E945E15C8CFBA
:107A90000E94D51582E20E9426151093720481E29D
:107AA0000E945E1580916804882309F4A1C082E0D9
:107AB0000E944215F9CE809166048F5F8093660420
:107AC000809166046E2D0E94A1459093660480917A
:107AD0006604F601E80FF11DF08082E00E94261591
:107AE00011E087E10E940913882309F41ACF8091DD
:107AF00066046E2D70E090E00197860F971F0E943C
:107B0000C1458093660480916604F601E80FF11D7B
:107B1000F08080E00E94261511E086E10E94E012CC
:107B2000882309F404CF82E00E945E150E942A1780
:107B300087E10E94E012882309F4FFCE80E00E94D2
:107B40005E150E942A1786E10E94CA12882309F452
:107B5000FACE80E00E94B412882309F4F4CE80911A
:107B60009D058093660480916604F601E80FF11D7F
:107B7000F08011E0E8CE0E94D51582E20E94261521
:107B800081E08093720481E20E942615809168044E
:107B90008823C1F082E00E94421580916604F601BC
:107BA000E80FF11DF08011E0B0CE81E00E94332992
:107BB0004ECF84E00E9433298CCE8FE0F82E0FE068
:107BC00010E013CF82E00E945E15E7CF82E00E94B2
:107BD0005E158091C40660910507409121062091B1
:107BE00027060BE616E00E94372C1092680466CE3A
:107BF00082E00E945E1558CE81E00E9433293ACE81
:107C00000F2D10E00F701070F0CE3F924F925F92E8
:107C10006F927F928F929F92AF92BF92CF92DF929C
:107C2000EF92FF920F931F93DF93CF93CDB7DEB701
:107C3000C058D0400FB6F894DEBF0FBECDBF109233
:107C400067041092650482E08093640440912706E3
:107C5000B1E4CB2ED12CCC0EDD1E8BE696E0B60126
:107C60000E94AE3BE82E0E9479148091120788236F
:107C700009F42CC684E00E943329992444248824E2
:107C80005524AA24AA94BB24332433943E01089497
:107C9000611C711C0E9479141091AB061F30A9F071
:107CA000103108F088C0113009F4B8C2143009F45A
:107CB0004CC20E94592B882369F70E94282B0E94EE
:107CC00079141091AB061F3059F70E943929882387
:107CD00009F09BC40E94AB2A86E10E94CA12882345
:107CE00009F08AC489E00E94CA12882309F0D5C22B
:107CF0008AE00E94CA12882309F0C7C286E10E9466
:107D0000E012882309F0BDC289E00E94E0128823B6
:107D100009F0B3C28AE00E94E012882309F0A9C2E8
:107D20008DE00E94CA12882329F080916204882382
:107D300009F031C591E0991609F4DBC3A2E09A1667
:107D400009F4D3C3B3E09B1609F0B3CF30926804B3
:107D5000682D70E0842D992787FD9095860F971FD9
:107D6000850D911D0E94C145582EEE2099F020E00E
:107D700030E0F601E20FF31F852D820F682D0E947F
:107D8000A145D301A90FB11D8C9180832F5F3F4F77
:107D90002E1578F340912706C6016BE676E00E9427
:107DA0007D3B409127068BE696E0B6010E94AE3BF4
:107DB000E82E99247ECF113109F41BC1113108F44A
:107DC00080C0123109F075CF0E943929882309F04B
:107DD00056C40E94AB2A8CE00E94CA12882309F084
:107DE00077C38CE00E94E012882309F06DC38EE017
:107DF0000E94CA12882309F05DC38FE00E94CA1254
:107E0000882309F04DC384E10E94CA12882309F037
:107E10003DC385E10E94CA12882309F02DC388E082
:107E20000E94CA12882309F01DC38EE00E94E0124E
:107E3000882309F0EFC28FE00E94E012882309F046
:107E4000F2C284E10E94E012882309F0F5C285E1C4
:107E50000E94E012882309F0F8C288E00E94E01234
:107E6000882309F0FBC2992009F423CF30926804DB
:107E7000EE2009F48FCF860110C00E97F9F08F2DF8
:107E80008A21D8019C919B21892BF80181938F0134
:107E90008E2F8C198E1508F07DCF0E94E000F82EF1
:107EA00090E08F7090708D30910539F7E7EFFE22EA
:107EB0008F2D90E08F7090700E9709F7F7EFFF22EB
:107EC000DECF0E943929882309F09EC20E94AB2A86
:107ED0008CE00E94CA12882309F0E7C187E10E9462
:107EE000CA12882309F0ECC180E00E94CA128823DC
:107EF00009F0F1C18CE00E94E012882309F0F6C17C
:107F000087E10E94E012882309F0F9C180E00E9415
:107F1000E012882309F0FCC18EE00E94CA12882377
:107F200009F0FFC18FE00E94CA12882309F008C23D
:107F300084E10E94CA12882309F011C285E10E94DF
:107F4000CA12882309F01AC288E00E94CA12882344
:107F500009F023C28EE00E94E012882309F02CC2AF
:107F60008FE00E94E012882309F02FC284E10E9472
:107F7000E012882309F032C285E10E94E0128823D2
:107F800009F035C288E00E94E012882309F038C267
:107F9000992009F48ECE30926804E2E09E1609F42E
:107FA000D0C3F4E09F1609F446C4B1E09B1609F073
:107FB00003C4EE2009F4EECE860107C00F5F1F4F09
:107FC000802F8C198E1508F0E5CE0E94E000F82E67
:107FD000EFE1E81798F30E94E000D8012C916E2D94
:107FE0000E94A145F601E90FF11D80818C93208349
:107FF000E5CF0E943929882309F0F9C20E94AB2AF3
:108000008CE00E94CA12882309F0E8C28CE00E942A
:10801000E012882309F0DEC28EE00E94CA12882393
:1080200009F0CEC28FE00E94CA12882309F0BEC2B6
:1080300084E10E94CA12882309F0AEC285E10E9441
:10804000CA12882309F09EC288E00E94CA128823BF
:1080500009F08EC28EE00E94E012882309F084C2EB
:108060008FE00E94E012882309F05FC284E10E9441
:10807000E012882309F062C285E10E94E0128823A1
:1080800009F065C288E00E94E012882309F068C206
:108090008DE00E94CA12882329F08091620488230F
:1080A00009F043C0192D10FF04CE3092680411FD71
:1080B000EFC2EE2041F1860106C00F5F1F4F802FF7
:1080C0008C198E1500F50E94E000F82EBFE3B8175A
:1080D000A0F30E94E000F82E90E08F7090708D3039
:1080E000910509F404C30E9709F4FEC29F2D9A214D
:1080F000D8018C918B21982B9C930F5F1F4F802F61
:108100008C198E1500F3BEEF9B2240912706C60105
:108110006BE676E00E947D3B409127068BE696E079
:10812000B6010E94AE3BE82EC4CD892D80958270A9
:10813000B1E09B22982A8DE00E945E15192D91FCDA
:10814000A2C388240E942A17AECF0E94392988230F
:1081500009F07FC284E00E940913882309F072C2EB
:1081600085E00E940913882309F065C282E10E941C
:108170000913882309F058C281E10E94091388235A
:1081800009F04BC286E10E940913882329F08091EF
:108190006804882309F0EDC287E10E94091388234F
:1081A00029F080916804882309F0B2C28091AB065F
:1081B000843041F01092720482E00E945E1582E2E7
:1081C0000E945E1580911207882309F48AC180916C
:1081D0007104813009F06DCD109271040E947E28E7
:1081E000882309F466CD10926404C058DF4F0FB69F
:1081F000F894DEBF0FBECDBFCF91DF911F910F91DD
:10820000FF90EF90DF90CF90BF90AF909F908F90B6
:108210007F906F905F904F903F9008950E94392912
:10822000882389F48091AB06813011F0109272049A
:1082300080911207882309F027C20E947E28882394
:1082400009F437CDD0CF0E94D51582E20E942615C1
:108250001093720481E20E945E1580916804882365
:1082600009F4A6C282E00E94421581E00E94270222
:10827000D9CF8CE10E945E1553CD8BE10E945E1533
:1082800049CD82E00E945E153FCD8CE10E9426150B
:108290009F2C93944424439431CD8BE10E94261566
:1082A0009F2C939444244A9423CD8EE00E9426155B
:1082B0009924939487E10E94CA12882309F414CE6A
:1082C00080E00E942615F2E09F2E80E00E94CA12F4
:1082D000882309F40FCE82E20E942615E3E09E2E49
:1082E0008CE00E94E012882309F40ACE8EE00E94FE
:1082F0005E1587E10E94E012882309F407CE80E032
:108300000E945E1580E00E94E012882309F404CEEA
:1083100082E20E945E158EE00E94CA12882309F450
:1083200001CE84E00E94261574E0972E60E1A62E0F
:108330005FEEB52E8FE00E94CA12882309F4F8CDB3
:1083400083E00E94261544E0942E30E2A32E2FED08
:10835000B22E84E10E94CA12882309F4EFCD88E08E
:108360000E94261594E0992E80E8A82E0FE7B02EE3
:1083700085E10E94CA12882309F4E6CD81E00E94BB
:10838000261514E0912EB0E4AB2EAFEBBA2E88E0A8
:108390000E94CA12882309F4DDCD84E20E942615CA
:1083A000F4E09F2EEFE0AE2E70EFB72E8EE00E942D
:1083B000E012882309F4D4CD84E00E945E158FE09A
:1083C0000E94E012882309F4D1CD83E00E945E155B
:1083D00084E10E94E012882309F4CECD88E00E9457
:1083E0005E1585E10E94E012882309F4CBCD81E07F
:1083F0000E945E1588E00E94E012882309F4C8CD2F
:1084000084E20E945E15C4CD89E10E94261599245C
:1084100044245CCD84E00E945E158FE00E94E0124F
:10842000882309F40ECD83E00E945E1584E10E944A
:10843000E012882309F40BCD88E00E945E1585E1E7
:108440000E94E012882309F408CD81E00E945E15A5
:1084500088E00E94E012882309F405CD84E20E949E
:108460005E1501CD84E20E942615992493942FE095
:10847000A22E90EFB92ED9CC81E00E942615992426
:10848000939440E4A42E3FEBB32EC9CC88E00E9425
:1084900026159924939460E8A62E5FE7B52EB9CCF3
:1084A00083E00E94261599249394E0E2AE2E7FED9E
:1084B000B72EA9CC84E00E94261599249394A0E1BC
:1084C000AA2EFFEEBF2E99CC8EE00E945E158FCCB7
:1084D0008EE00E94261599249394AA24AA94BB2482
:1084E00080CC81E00E94332972CE442009F02ECC4A
:1084F000E0CB442009F4DDCB90926804EE2089F0B3
:10850000342D3E0DD60120E0822F830F6E2D0E9468
:10851000A145F301E90FF11D8D9180832F5F2E1589
:1085200098F340912706C30138CC83E00E945E1582
:1085300084E10E94E012882309F49ECD88E00E9425
:108540005E1585E10E94E012882309F49BCD81E04D
:108550000E945E1588E00E94E012882309F498CDFD
:1085600084E20E945E1594CD84E00E945E1578CD71
:1085700084E20E942615A1E09A2A1FE0A12EB0EF06
:10858000BB2E68CD81E00E94261591E0992A80E4F7
:10859000A82E0FEBB02E58CD88E00E94261581E062
:1085A000982A20E8A22E9FE7B92E48CD83E00E94AA
:1085B0002615F1E09F2A40E2A42E3FEDB32E38CDE0
:1085C00084E00E942615E1E09E2A60E1A62E5FEE7F
:1085D000B52E28CD8EE00E945E151ECD8EE00E9445
:1085E0002615B1E09B2AAA24AA94BB240FCD8CE0C7
:1085F0000E942615992402CD82E00E942615409003
:108600009D054194992493946DCB80E20E94261598
:1086100099244424FF2455245DCB6091AB0681E16D
:1086200041E10E941F29AECD6091AB0682E142E19B
:108630000E941F29A1CD6091AB0680E145E00E9418
:108640001F2994CD6091AB068FE044E00E941F2962
:1086500087CD0E94D51582E20E94261530927204C1
:1086600081E20E94261580916804882309F47DC068
:1086700082E00E94421581E00E9427026BCD8BE0D0
:108680000E9426159924A5CB84E00E943329D5CDDC
:10869000EE2009F438CD860107C00F5F1F4F802FF1
:1086A0008C198E1508F02FCD0E94E000F82EEFE314
:1086B000E81798F30E94E000682D0E94A145F3019D
:1086C000E90FF11DF0808F2D90E08F7090708D304C
:1086D0009105B9F00E9791F09F2D9A21D8018C91B8
:1086E0008B21982B9C93D9CFF7EFFF22FFCCE7EF9C
:1086F000FE228F2D90E08F709070F5CC87EFF822DE
:10870000EBCFF7EFFF228F2D90E08F709070E2CFCC
:1087100082E00E945E158091C40660910507409139
:108720002106209127060BE616E00E94C22B4091FD
:108730002706C801B6010E94AE3BE82E10926804DD
:1087400035CD8E2D869509F425CBD6016E2D615041
:10875000262F281B8C91F601E60FF11D90819D9329
:10876000808361506217B1F715CB82E00E945E15DD
:1087700082CF82E00E945E158091C4066091050759
:1087800040912106209127060BE616E00E94372C27
:108790001092680401CDF39481E0F8228DE00E94EC
:1087A0005E15FF2009F07BC088240E942A17C2CAE8
:1087B00082E00E945E1559CD609127068BE696E017
:1087C000A6012FE935E00E944129E82E882311F106
:1087D000860106C00F5F1F4F802F8C198E15D0F4B5
:1087E0000E94E000F82EBFE3B817A0F30E94E0005B
:1087F000F80120816E2D0E94A145F601E90FF11DBF
:108800008081D8018C9320830F5F1F4F802F8C199C
:108810008E1530F3609127068BE696E0A6012FE9CE
:1088200035E00E94222A409127068BE696E0B601A9
:108830000E94AE3BAFCAEE2009F4ACCA860107C065
:108840000F5F1F4F802F8C198E1508F0A3CA0E944E
:10885000E000F82E8FE38F1598F30E94E000D80116
:108860002C916E2D0E94A145F601E90FF11D80812A
:108870008A219B2D9223892B8C9380818B212A2105
:10888000822B8083DDCF8DE00E94261581EE95E05E
:10889000B301409162040E94AE3B882E53CC8DE020
:1088A0000E94261581EE95E0B301409162040E947A
:1088B000AE3B882E409127068BE696E0B6010E94DB
:1088C000AE3BE82EA3E09A2E44246FCF81E00E94B5
:1088D0003329D3C9EF92FF920F931F930E9479140B
:1088E00080911207882309F428C184E00E9433296B
:1088F000FF24F39407C0113009F472C00E94592B71
:108900008823C9F00E9479141091AB061330D9F076
:10891000143088F31430E9F11D3081F781E00E94B2
:1089200039308091AB068D3049F3109272040E9469
:10893000592B882339F70E94282B0E947914109113
:10894000AB06133029F70E943929882309F0B2C0F9
:108950000E94AB2A882321F01092640410927204C2
:108960000E945F13882309F092C080911207882328
:1089700029F686E10E94CA12882309F0D3C086E155
:108980000E94E012882309F4B9CF80E00E94A91C5C
:10899000B5CF0E943929882309F0A0C080E00E9449
:1089A0003930882309F497C08091AB06843011F0E8
:1089B0001092720480911207882309F4ABC0809151
:1089C0007104813009F09ACF109271040E947E28C0
:1089D000882309F493CF1F910F91FF90EF90089592
:1089E0000E9439298823B9F580E00E943930182F78
:1089F00086E10E94CA12882319F586E10E94E012DE
:108A00008823D1F41123A9F08091AB06813011F0B5
:108A10001092720480911207882309F07FC00E948F
:108A20007E28882309F46ACF1F910F91FF90EF9061
:108A300008950E94462BE8CF80E00E94A91CE2CF57
:108A400080E00E9417299091B306890F60E040E012
:108A50000E94921CD2CF0E94D51582E20E94261558
:108A60001093720481E20E945E158091210660914C
:108A7000270640919A052091280600912106E09052
:108A800098050E94191881E00E942702ADCF182F87
:108A900011500E940A17812F0E94E1161093AC0614
:108AA00080911207882309F060CF8091AC068093F3
:108AB000B3065BCF0E94D515F092640481E00E945A
:108AC000270284E20E9426158091AC060E94E116DE
:108AD000F09272043DCF0E94462B66CF0E94D515BE
:108AE00082E20E942615F092720481E20E9426150D
:108AF000809121066091270640919A0520912806D1
:108B000000912106E09098050E94191881E00E94CA
:108B1000270244CF81E00E94332951CF84E00E9494
:108B200033297DCF80E00E9417299091B306890FE9
:108B300060E040E00E94921C22CF81E00E94332935
:108B4000D7CE991B79E004C0991F961708F0961BA1
:108B5000881F7A95C9F780950895AA1BBB1B51E120
:108B600007C0AA1FBB1FA617B70710F0A61BB70B9D
:108B7000881F991F5A95A9F780959095BC01CD0142
:108B8000089597FB092E07260AD077FD04D0E5DF6C
:108B900006D000201AF4709561957F4F0895F6F77E
:108BA000909581959F4F0895A1E21A2EAA1BBB1B99
:108BB000FD010DC0AA1FBB1FEE1FFF1FA217B307A9
:108BC000E407F50720F0A21BB30BE40BF50B661FBF
:108BD000771F881F991F1A9469F760957095809583
:108BE00090959B01AC01BD01CF010895F894FFCF92
:108BF000010001000100010001000100010001006D
:108C00000100010001000100010001C000800040DE
:108C1000007F206430480F04050607111210130E60
:108C200004050607111210130409050A06070B11A3
:108C30000C120D101325212326272422201D1E1B74
:108C4000191F1C1A1012180F110C130E0B140D0AF9
:108C50001516091704050803060107000203201969
:108C60001A180C0B0A090420191A180C0B0A0922ED
:108C700021252320191A18241B1C0F0E0D04030A8A
:108C80000C0B0908010200201B191C1A180F0C0EEE
:108C90000B0D0A0926271D1E1F101211131415167D
:108CA000170506076E306E783078000100070E0950
:108CB0001C1B1215383F363124232A2D70777E79FC
:108CC0006C6B6265484F464154535A5DE0E7EEE9EC
:108CD000FCFBF2F5D8DFD6D1C4C3CACD90979E99DC
:108CE0008C8B8285A8AFA6A1B4B3BABDC7C0C9CECC
:108CF000DBDCD5D2FFF8F1F6E3E4EDEAB7B0B9BEBC
:108D0000ABACA5A28F88818693949D9A2720292EAB
:108D10003B3C35321F18111603040D0A5750595E9B
:108D20004B4C45426F68616673747D7A898E87808B
:108D300095929B9CB1B6BFB8ADAAA3A4F9FEF7F07B
:108D4000E5E2EBECC1C6CFC8DDDAD3D4696E67606B
:108D500075727B7C51565F584D4A4344191E17105B
:108D600005020B0C21262F283D3A33344E4940474B
:108D700052555C5B7671787F6A6D64633E3930373B
:108D800022252C2B0601080F1A1D1413AEA9A0A72B
:108D9000B2B5BCBB9691989F8A8D8483DED9D0D71B
:108DA000C2C5CCCBE6E1E8EFFAFDF4F30409050A0D
:108DB00006070B110C120D10130001000100010039
:108DC000010001000100010001000100010001009B
:108DD000010001C000800040000606011718191AA2
:108DE0001B1C1D1E1F202122233F3F3F0B0C0D0E7D
:108DF0000F10111213141516173F3F3F2324252679
:108E00002728292A2B2C2D2E2F3F3F3F1718191AC0
:0E8E10001B1C1D1E1F202122233F3F3F15006B
:00000001FF
